:020000040800F2
:10500000101E00208151000865960008E98C0008F8
:105010000000000000000000000000000000000090
:10502000000000000000000000000000B5A400081F
:105030000000000000000000359E0008F1A50008F7
:1050400093510008935100089351000893510008B0
:1050500093510008456700089351000893510008D8
:1050600000000000935100086D660008935100088D
:10507000935100084D920008000000009351000871
:105080000000000093510008000000000000000034
:10509000935100080000000093510008935100084C
:1050A00093510008935100089351000821B1000862
:1050B0009351000893510008000000000000000018
:1050C00000F002F800F030F80CA030C808382418BE
:1050D0002D18A246671EAB4654465D46AC4201D130
:1050E00000F022F87E460F3E0FCCB6460126334232
:1050F00000D0FB1AA246AB46334318476473000046
:10510000847300000023002400250026103A01D3F8
:1051100078C1FBD8520700D330C100D50B6070476F
:105120001FB51FBD10B510BD01F088F91146FFF77E
:10513000F7FF06F065FE01F0A0F903B4FFF7F2FFF8
:1051400003BC01F0D1F9000070B505460C461646C7
:1051500002E00FCC0FC5103E102EFAD2082E02D35B
:1051600003CC03C5083E042E07D301CC01C5361F6E
:1051700003E021782970641C6D1C761EF9D270BD85
:105180000748804707480047FEE7FEE7FEE7FEE7DF
:10519000FEE7FEE704480549054A064B7047000054
:1051A0008DA60008C150000810180020101E002015
:1051B000101A0020101A0020FEB5054610460C46B5
:1051C000184373D0AE468C460020AD1A01469C4170
:1051D00067D36646002701243D46B61A9D4102D397
:1051E00013463A462124654676462F04360C3E4344
:1051F0002D0CB61A9D4104D3150C1B042B4312042D
:105200001034654676462F06360A3E432D0AB61AF6
:105210009D4104D3150E1B022B4312020834654630
:1052200076462F0736093E432D09B61A9D4104D311
:10523000150F1B012B431201241D65467646AF074F
:10524000B6083E43AD08B61A9D4104D3950F9B00A6
:105250002B439200A41C65467646EF0776083E4332
:105260006D08B61A9D411AD392185B41641C16E072
:105270000018764665464941B71A9D410191009054
:1052800009D36046B11A98418E4684460098019928
:105290000025401C6941DD0752082A435B08641E53
:1052A000E6D57246634603B0F0BDFFE70020014635
:1052B000C046C0462A462346F5E7034610B50B43D1
:1052C0009B070FD1042A0DD308C810C9121FA3428F
:1052D000F8D018BA21BA884201D9012010BD0020A7
:1052E000C04310BD002A03D0D30703D0521C07E0EF
:1052F000002010BD03780C78401C491C1B1B07D1F3
:1053000003780C78401C491C1B1B01D1921EF1D163
:10531000184610BDF8B5042A2CD3830712D00B7899
:10532000491C0370401C521E83070BD00B78491C8C
:105330000370401C521E830704D00B78491C037075
:10534000401C521E8B079B0F05D0C91ADF0020237B
:10535000DE1B08C90AE0FFF7F7FEF8BD1D4608C9C5
:10536000FD401C46B4402C4310C0121F042AF5D245
:10537000F308C91A521EF0D40B78491C0370401C64
:10538000521EEAD40B78491C0370401C012AE4D455
:1053900009780170F8BD01E004C0091F0429FBD29F
:1053A0008B0701D50280801CC90700D002707047AE
:1053B00000290BD0C30702D00270401C491E0229ED
:1053C00004D3830702D50280801C891EE3E70022F4
:1053D000EEE70022DFE7002203098B422CD3030A09
:1053E0008B4211D300239C464EE003460B433CD432
:1053F000002243088B4231D303098B421CD3030A9A
:105400008B4201D394463FE0C3098B4201D3CB01C9
:10541000C01A524183098B4201D38B01C01A5241F9
:1054200043098B4201D34B01C01A524103098B42FD
:1054300001D30B01C01A5241C3088B4201D3CB00E8
:10544000C01A524183088B4201D38B00C01A5241CB
:1054500043088B4201D34B00C01A5241411A00D27B
:1054600001465241104670475DE0CA0F00D04942E4
:10547000031000D34042534000229C4603098B4254
:105480002DD3030A8B4212D3FC22890112BA030ADC
:105490008B420CD3890192118B4208D3890192115E
:1054A0008B4204D389013AD0921100E08909C309E3
:1054B0008B4201D3CB01C01A524183098B4201D3E5
:1054C0008B01C01A524143098B4201D34B01C01AD0
:1054D000524103098B4201D30B01C01A5241C30848
:1054E0008B4201D3CB00C01A524183088B4201D3B7
:1054F0008B00C01A5241D9D243088B4201D34B00D2
:10550000C01A5241411A00D20146634652415B1013
:10551000104601D34042002B00D5494270476346F4
:105520005B1000D3404201B50020C046C04602BD1A
:1055300070477047704700000246C80FC00781439C
:105540004B0030B54B405B009B0D20D01923DB0690
:10555000C91801231B05994220DB0324A407042555
:105560001346AB400BD3002B04D1EB0613409B003A
:10557000E34204D401246407002312195941FF2394
:105580001B0599420BD2C9000143500F09E0CB0221
:1055900004D501430803024305D0054830BDFF216F
:1055A000C905084330BD084607210905884330BDB9
:1055B0000000C07FF0B50C46871A9C410D46861A44
:1055C0009D4103D2C01BA141D21963410D0D1F0D96
:1055D000C94EEC1BAE435CD07F057F0D0026002F2B
:1055E00051D02D05AC46A943DD020123ED0A1B0570
:1055F0001D4320231B1B24D41746E7403818714154
:105600002F46E740CC199D402818314661410C0DCA
:1056100027D161449A4013D50023401C59415200C0
:105620000ED14008400001224B005205D34207D35F
:1056300005204007C14201D5B04900E0B0493046DD
:10564000F0BD6B00002A00D001229A181F23203CD5
:105650001B1B01D5002302E0E540281871410C0D09
:10566000D7D0012424050919C407CD0740084908EB
:10567000E40F28436144002CD5D00024401C614134
:105680009A40D0D1CDE76A05520DD9D1C90FC907CB
:10569000D5E79C4D4E00002801D0012400E00024F5
:1056A00034195F00002A01D0012600E00026BE194F
:1056B000954FAC420CD8AE420AD8B44206D0012570
:1056C0006D05EC42BCD010461946F0BD9942FCD0A5
:1056D00000203946F0BDF0B51FB40C460F46811AC4
:1056E0009F412546861A9D4106D20125ED076F4050
:1056F000401ABC4152187B41210D1E0D8D1BAC463A
:105700007D4D8D437ED075056D0D7CD00D05AE466B
:10571000AC431B031B0B794D52429D41202366462F
:105720009B1B14D31746F74038180026009074418D
:1057300060462F460741E41900989D4028186641AD
:1057400016D4714671189A4025D5012320E093188C
:105750002A466A415200002B00D0521C1E23203ED4
:105760009B1B002B61DD3541EE1728186641E8D5FB
:10577000001876415B1C9A4000D3401C4B05F3187F
:105780001524E34010D3002B52D071467118D30F6B
:10579000C01802D3491C05B0F0BD0123DB079A42B3
:1057A000F9D140084000F6E701225205B21801D1B4
:1057B000002853D00123CC0ADB029943891E002A1A
:1057C00008D1020C03D0020C0004103902E002469A
:1057D000002020390023550B05D112020823550B58
:1057E00001D152010D23550C01D112011B1DD50C05
:1057F00001D192009B1C150D01D152005B1C20258C
:10580000EE1A01E02CE022E00546F54015439840F1
:10581000CA1AE10769181305C918002ABBDA032060
:1058200040070818C10FC9070FE071466118B2E7B9
:10583000F10740080843711071444A000CD001235D
:105840005B059A42A7D2C90FC9070020A3E7490503
:10585000490D26D1002001E00028F4D100219AE76B
:10586000284D6600002801D0012100E000217118B8
:105870005F00002A01D0012600E00026BE19224F59
:10588000A94210D8AE420ED8B14208D001256D050C
:10589000E94206D01946A802414010467BE79C42E7
:1058A00001D0214677E70020394674E710B50C4651
:1058B0005C4005D50124E4076340FFF70CFF10BDF1
:1058C000FFF778FE10BD30B40C465C4004D50124CF
:1058D000E407634030BC6DE630BCFCE670B50124E3
:1058E000E40761400D465D4002D4FFF763FE70BDE2
:1058F0006340FFF7F0FE70BDFF0700000000F0FFFF
:105900000000F07F0000E0FF0000F87FF0B5F94DE7
:105910000C091E092C402E402F468BB0A7437DD08A
:10592000B543FCD0002E7AD0002CFCD00D465D4053
:10593000ED0F2543AC1BFF25AD0464190894C50287
:10594000440DC9022143500DDC0204430120C0076D
:1059500001430443D2020191200C110C00958C46A6
:10596000010423468B430A9161460904E24D8A43B0
:105970000991010A7D4449198039097805464D434A
:1059800001266D18F605751B6943C90C640B891C4B
:105990004C436418B5012C1B250C2E04B4434C4316
:1059A0004D43210C691889090591009DE90701D033
:1059B0000121C90704912C4601996708CD072F439F
:1059C0004C08059DE10B4D432D0C29466646754359
:1059D00002950D4645432E46029D7D1BB441009520
:1059E0000D465D4301942C0C2F040D465543AE46E5
:1059F0002D0C3D43029503947546049C2D04641BB5
:105A0000049406D2029C039D641C002675410395F4
:105A1000029401AC70CC009F7D1B01E03EE162E18D
:105A2000B44109040095079101940599A4086143C4
:105A3000090C0C464443650BE7040C466646744368
:105A4000A646640B3C43039502947446049DE4040B
:105A50002C1B049406D2029C039D641C00267541F5
:105A60000395029401AC70CC009F7D1BB44101945E
:105A70000C465C430095650FE7000C465443A64670
:105A8000640F3C43039502947446049DE4002C1B70
:105A9000049406D2029C039D641C00267541039564
:105AA000029401AC70CC009F7D1BB441AE09AF06DF
:105AB000049DC900AD092F43049DA406AD060495BD
:105AC000079D344369180791059DE10B4D432D0C4B
:105AD00029466646754302950D4645432E46029D6E
:105AE0007D1BB44100950D465D4301942C0C2F04A1
:105AF0000D465543AE462D0C3D4302950394754625
:105B0000049C2D04641B049406D2029C039D641C17
:105B1000002675410395029401AC70CC009F7D1B5B
:105B2000B44101948C050694079C890A611800957C
:105B30000791019C0599A4086143090C0D46454352
:105B4000680BEF040D46644665436C0B3C43049FB1
:105B5000ED047D1BAC4602D20025641C6841009E0A
:105B6000019D371B85410846584301950C46460F59
:105B7000C5005443600F28436546E4002C1B02D245
:105B80000025401C6E41019D3F1AB5412846BD09C4
:105B9000800628438446A009BF064E020699A40643
:105BA00076180743079D002068410A99079019431A
:105BB0000020099B00906046FF1913434041E20F0B
:105BC00064003A43A4460446D71A8C41A04203D944
:105BD0000120009020463A46C70F94184041624683
:105BE000D20F2243644664000494009CBE466400C5
:105BF000D71AA446044602978C417746002F01D15C
:105C0000A04204D96046401C8446029A2046C40F34
:105C1000A64694184041049A0546D20F2243644692
:105C20006400D31A8D417146002901D1A84202D9DE
:105C300028461A46641C10430122002800D016434F
:105C400061020020079B891904465C410223002C55
:105C500002DB491813466441089DCE0A2D145D19D4
:105C60004B056705E10A2C050D1908993E43C90744
:105C70006940002B08D0934006D30022761C514186
:105C8000002B01D1760876001C4A002D43DB15421B
:105C900041D0AA433FD030460BB0F0BD06180D46A8
:105CA0004D41174C7642AC411AD395181C465C41C5
:105CB000134A6D42A24113D3012252054C00D44233
:105CC0000AD15C00D4420BD04B4002D59202114362
:105CD000E2E749004908DFE75940C90FC90718E062
:105CE00000200849D8E7054801420DD10342F7D00A
:105CF000F2E700000000FF07276A00000000F07FC5
:105D00000000E0FF0000F87F114859400143C01235
:105D100041400020C0E70123089A9B069A4205DC17
:105D2000032252078918C90FC907B5E70522520790
:105D30008918074A1143D2125140ADE770B5154694
:105D40001C4602460B4628462146FFF7DFFD70BD84
:105D5000FFFFFF7F30B50346CA02400D1043164DCA
:105D6000164C0A1502D02043002A06DBAA1A002A84
:105D700012DDD040FF2A0BDC30BD5205520D01D19F
:105D800040004008AA1A07D4D0404042FF2A01DD53
:105D9000002030BD0028FCDD4A00002B01D001208E
:105DA00000E00020101801225205D042F0D8C81798
:105DB000C043604030BD00001E04000000000080B1
:105DC0000346CA02400D10B510430A1504D0012441
:105DD000E4072043002A05DB0A4CA21A04D4D04071
:105DE000FF2A00DD002010BD4A00002B01D0012059
:105DF00000E00020101801225205D042F2D8C81746
:105E0000C04310BD1E0400001F22030C02D10F224C
:105E1000000402D0030E03D004E0002001467047C6
:105E20000002083A030F01D10001121F830F01D1B4
:105E30008000921E002801DB4000521E12055118FE
:105E40004205C012411810467047C10FC90700D063
:105E50004042012292071143D6E701218907D3E787
:105E6000F0B58B4C0F09254689B0BD437BD01D0989
:105E70002646AE43FAD00E465E402740F60F3E431C
:105E8000254071D024012142FBD0FF24AD19A40488
:105E90002D1B039501252D05DB02DB0AC9022B43CF
:105EA000C90A29431E010901040F130F05012143EB
:105EB0001701880B820391432D098C46A90B1E43C1
:105EC0008A039543B30B9A0396433F09BA0B940395
:105ED000A74302962E467E430497B6464E19D7191D
:105EE0000C460196544305977E43371B7646BF1BED
:105EF0003601B646BE0B361900967646BC043719F5
:105F0000009C01D3641C00946400002F01D0012682
:105F10003443029E049F754366467E430496760092
:105F200034196E0034190094029C019E1C196643BA
:105F3000751BAE46069465464519059C05956C4350
:105F4000594375460891691A0191049E01465143CF
:105F5000A41B0491611A009C0791E10605D0610918
:105F60000122114302E072E06EE06109089D002702
:105F70002C0A2D066918049D7C412A0A2D066918F1
:105F8000019D6241AC0DAD026D185441079A910D0F
:105F9000920255196141029A644658435443069B44
:105FA000059A5A43121A131B9A0E9B015B187A41E9
:105FB000010B0005C3185141220A200644195A4119
:105FC0009A4200D2491C01204002814203D315238A
:105FD0000226F64302E014230326F6432020C51AC6
:105FE000A9401746AF40DA400A4320460399D840FB
:105FF0000914731819055118039A3843D2075140F0
:10600000AC4009D00122944006D30022401C5141EB
:10601000002C01D1400840001E4A934212D30122B5
:1060200003989206904207DB0520400709181A489A
:106030000143C012414004E0032040070818C10F8B
:10604000C907002009B0F0BD0020F107FAE70518E4
:106050000C464C4111486D42A04115D394181A4684
:106060005A410E48644290410ED301204A00400537
:10607000824209D35A00824206D35940C90F084AC6
:10608000C90700201143DDE700200649DAE70000D8
:106090000000FF07FE070000FFFFFF7F0000E0FF9A
:1060A0000000F07F0000F87F0121C905012341189D
:1060B00042001B06D3185B0E0AD0C1100722D2067D
:1060C000891840075242D14201D5520089187047C1
:1060D000090208D50146002A03D0C10FC9070020D4
:1060E000704710467047420202D0002002497047B4
:1060F000072109050143F4E70000F87FF0B5FF250B
:106100002D04C609C209FF2704462E400137CB09DA
:106110003E4348402A402B400746002A6BD0002BC4
:1061200069D0AA4267D0AB4265D0002800DA324677
:106130000125ED0529432C4309022002090AD21A40
:106140004B0C7F24E31A434C000A7C44E35C7D241F
:106150002404121914145B00A218884201D3521CA3
:1061600000E0400049420C465C4324115C43DB01E3
:106170006415E318040A5C43C502200D0C46444331
:106180006419250A5D432303EC0C0D4665430003A7
:106190000019EB184C42A34201D35B18401CD405F4
:1061A0002018002B07D05B00C91804D3401C00291D
:1061B00001D1400840003F2189048A4209D3002AC6
:1061C00008DC1106090F04D0032149074018C00F4D
:1061D000C007F0BD01224100120689187F22520635
:1061E0009142F6D205214907C84201D59010F0BD71
:1061F000FF20C005F0BD002F00DA32461648AA4243
:1062000007D2AB4205D21902090E17D0F80FC0070A
:10621000F0BDFF2563002D06AB42F9D84900A94225
:10622000F6D8AB4201D1A942F2D0A94201D1002156
:1062300001E061004908D0050843F0BD1102090ED4
:10624000FBD0FF200243D005F0BD0A4601461046B0
:1062500054E70000D16200000000C07F0102C215B7
:1062600004D00123DB071943002A0ADB9E239A1A74
:1062700002D40846D0407047FF22410012069142E6
:1062800001D900207047C017C04370471F22030C7C
:1062900002D10F2200041CD0030E01D10002083AE3
:1062A000030F01D10001121F830F01D18000921E44
:1062B000002801DB4000521ED2055118021251186D
:1062C0001922904004D3491C002801D149084900F3
:1062D00008467047C10FC90700D04042012292070B
:1062E0001143D3E701218907D0E70000F8B5224C1C
:1062F0004E00069DA6420AD8A64201D1002806D12A
:106300005E00A64203D8A6420AD1002A08D00D2476
:10631000240425422CD02946002000F061F8F8BD65
:106320000C461C430CD4994202D0EFF30080F8BD18
:10633000904202D0EFF30080F8BDEFF30080F8BD8B
:1063400009242407E5008B4206D0EFF30080A04328
:10635000591A06D2284304E0101A05D3EFF300803F
:10636000A04380F30088F8BDEFF30080A043F1E77D
:10637000009500F04DF8F8BD0000E0FF10B5FF23D8
:106380001B0644009C421DD84C009C421AD8034670
:10639000124A0B4307D4401A02D3EFF3008010BD1A
:1063A000EFF3008010BD081A06D2EFF30080012140
:1063B0009043C907084302E0EFF30080904380F365
:1063C000008810BD0D231B041A4204D01146002082
:1063D00000F006F810BD00F025F810BD0000009098
:1063E000C80212D54803400F002804D0C803C04398
:1063F000012188407047EFF300800001000903216C
:106400000907084380F300887047002070470000A8
:1064100010B500200249029A00F037F810BD0000C4
:106420000000F87F10B5024800F02FF810BD000002
:106430000000C07F00487047AC1700207546FFF78A
:10644000F9FFAE46050069465346C008C0008546C0
:1064500018B020B5FEF79EFE60BC00274908B6467E
:106460000026C0C5C0C5C0C5C0C5C0C5C0C5C0C563
:10647000C0C5403D49008D46704710B50446C04632
:10648000C0462046FEF759FE10BD10B50C46110758
:10649000090F092904D00A290AD008290CD104E0DF
:1064A00011460820FFF79CFF06E0510606D501E0E3
:1064B000510601D50120C007214610BDD10607D5E0
:1064C00001010909CC084907000E0006044309E050
:1064D000410F20024907000A0143200E00061D2239
:1064E000D14101430846E7E701491820ABBEFEE76A
:1064F00026000200704770B58C180578401C6B07A9
:106500005B0F01D10378401C2A1106D10278401C90
:1065100003E00678401C0E70491C5B1EF9D12B0766
:1065200005D40023521E0DD40B70491CFAE70378E2
:10653000401CCB1A921C03E01D780D70491C5B1C9B
:10654000521EF9D5A142D8D3002070BD38B50446FB
:10655000064805490068FEF73EFF604300E0401E24
:1065600000900028FBD138BD40420F006C01002094
:10657000F8B50446006881688907890F012902D1AE
:106580000168C90727D18168144A102611400125E6
:10659000002913D18168294381600120FFF7D6FFCC
:1065A00001F024F8074611E001F020F8C01B0A288A
:1065B0000CD920680068C043C00707D0606D304325
:1065C0006065A06D2843A0650120F8BD20680068C3
:1065D000C043C007E8D10020F8BD000017000080CC
:1065E00070B51848808F00282BD0174C0125A66A5B
:1065F000ED05AE4201DA30460BE0208AFFF772FE6D
:1066000001467F20C005FFF779FD314605F0FEFD0C
:10661000A062A84208DBA078002805D104210B481D
:1066200002F0CEF80120A070A06AA84209DAA07892
:10663000012806D10020A070A0620421034802F0C6
:10664000FDF870BD9C0D00202401002040160020A4
:1066500010B500231A4603E0845CE3189BB2521C79
:106660008A42F9D3D84380B210BD000010B5034868
:1066700000F05CFD024800F059FD10BD4C170020F1
:106680000417002030B5446C1C252C400125A54082
:10669000046C6560046863608368102B036803D032
:1066A00099600068C26030BD9A600068C16030BD0A
:1066B0001449012048720A4602205E3250720320BB
:1066C0003C3A507204200E3A50720F480D4B00783D
:1066D000087022310870203108770C495A1C08785C
:1066E000587149789971233318715971203318778B
:1066F0005977107551751A461E32107551751076FE
:10670000517670479C11002027010020480100208D
:1067100010B503F0A5FE202003F060FF012005F076
:10672000D5F8002003F05AFF044804F073FF044832
:1067300005F022FA002005F057FA10BDE80000200D
:106740008380000070B503F057FF0520012100078A
:1067500000F038FF00250E4C002800D065600221B3
:106760000C4800F02FFF00280AD1012020700A48B1
:10677000808F002803D001200849800708606560E9
:10678000012000F03BFE022000F038FE70BD00004A
:1067900058010020000400509C0D00204C010020F6
:1067A0007047000010B5084900224A6107494B684C
:1067B0004C1523434B604B68082423434B60C009AE
:1067C000C001026010BD00009417002000200240AC
:1067D0007FB500250C460646039500F0DFFDE00975
:1067E000029003A901960095684600F06FFD00280D
:1067F00004D000F0A7FD002004B070BD00F0A2FDA1
:106800000120F9E710B5002302E0C45CCC545B1C06
:106810009342FAD310BD000010B5214A00219069BF
:10682000C305204804D541690223194341619115EC
:1068300093699B0505D543690124234343616302A2
:10684000194393695B0505D54369082423434361D4
:10685000E301194393691B0505D5436904242343C8
:1068600043616302194393699B0405D5436910246E
:10687000234343616302194393699B0304D544692D
:1068800020231C43446119439369DB0305D5436905
:10689000402423434361A0020143916110BD0000E5
:1068A000002002409417002070B5054600F09EFEBF
:1068B0000646184C0AE0681C08D0002D04D000F0F1
:1068C00095FE801BA84201D9032070BDA069C007B6
:1068D000F1D1A069800701D50220A061A069C0059F
:1068E00011D4A06980050ED4A06940050BD4A0691D
:1068F000000508D4A069800405D4A069800302D4EF
:10690000A069C00303D5FFF787FF012070BD0020F9
:1069100070BD000000200240F8B51746002605466D
:106920000C4600F03BFD09E029460220226800F0F9
:1069300017FD002804D1241D2D1D361DBE42F3D3A2
:1069400000F000FDBE4201D20020F8BD0120F8BDDC
:1069500010B5084902460020054B497905E044007E
:106960001C5B944203D0401CC0B28842F7D310BDD8
:10697000401300205800002010B500F028FE10BD84
:1069800010B5094801F046F880B2FFF766FA074AE9
:10699000074BFFF765FA0022064BFEF7B7FFFFF73C
:1069A0000FFA80B210BD0000B8150020F853E3A51F
:1069B0009B843E4000408F4070B50024204603F089
:1069C000D1F947494748A200641CE4B28150142C15
:1069D000F9D3464944480A790275497941754449D1
:1069E0000A780276497841763F490520133148728A
:1069F0000A2005F0B1F87D20400105F0C7F83A49BA
:106A0000002213310C2005F091F900210C2005F033
:106A10009FF9384800F0FEFF344C0125223C2085C8
:106A2000AD0309E0334800F0F5FF80B22085E18E28
:106A3000FF392D39884206DBE18E80B28842F1D3DE
:106A400049198842EED8022005F0D6F8002003F05C
:106A500089F9294D00210F2004F0FEFF284220640F
:106A6000F8D0206C411C38D0400435D58122D201A9
:106A700000210F2005F02FF90021102004F0ECFF79
:106A800041061948490E0022C73005F01BF8164D83
:106A9000C735687A05281FD102221549681DFEF7FF
:106AA0000CFC002818D11148AE7C66710422691CC8
:106AB0003630FEF72FFC29461331084672000D468A
:106AC0006930FEF727FC60792946420005484838BE
:106AD000FEF720FC0320207070BD04F013FC0000C2
:106AE000FFFF0100A0130020FD1100207A0000200C
:106AF00048010020B815002000D0272410B5084810
:106B000000F09EFA0A21064800F036FA044800F028
:106B100021F9800503D5024800F01EF980B210BDAE
:106B20005C150020F8B52F4D00220121284600F009
:106B300056FDFFF7E3FFFFF7D5FB2B4E3146FFF77E
:106B4000DDFA2A4C0122A0601146284600F047FDDC
:106B50002749A068002588423EDB2078254F002881
:106B600015D02570FFF7CAFFFFF7BCFB3146FFF7D2
:106B7000C5FAA060FFF798FA00223B46FEF7A3FE95
:106B800000221D4BFFF76CF9FEF7D6FC6060A06891
:106B9000FFF78AFA00223B46FEF795FE174A184B8C
:106BA000FFF75EF906460F466068FFF77DFA134A65
:106BB000144B5242FFF754F932463B46FEF776FE3D
:106BC000FEF7BAFC10496060884201DD616004E0B4
:106BD000FF21C905C84200D365606068FFF73EFB2E
:106BE000C0B2F8BD0004005000401B44300000203B
:106BF0000000604000000C4000E064403333333359
:106C000033B33040CCCCEC3F0000C842F8B5054669
:106C100004464035287C0026012808D0012028742D
:106C2000206881688907890F01290ED101E00220BF
:106C3000F8BD0168C90708D0606D20210843606570
:106C40000126002028743046F8BD616DFF22013214
:106C50009143022211436165C1688907890F009140
:106C6000C16889088900C160206881689207114362
:106C7000816000F0BBFC074612E000F0B7FCC01BCF
:106C80000A280DD920688068002809DA606D022181
:106C90008843102108436065002028740120F8BD56
:106CA000206880680028E8DB2068C168009A1143EA
:106CB000C160606D80088000401C6065C1E7000015
:106CC000F8B506460D464036317C01290DD001212C
:106CD000317401688A68520709D5416D2022114339
:106CE0004165002030740120F8BD0220F8BD174B2B
:106CF0006A68D80547109A42154C8A6A2B6812D0E8
:106D00005B035B0B1A438A622968490305D5A168B6
:106D10000143A1600A20FFF719FC2868800312D5FF
:106D2000A06838430EE05B035B0B9A438A622968D4
:106D3000490302D5A1688143A1602868800302D578
:106D4000A068B843A06000203074F8BD01100000B6
:106D500000270140406D70470068006C70470000DC
:106D600070B5040006D0606D264600254036002828
:106D700002D006E0012070BDA5653574204600F004
:106D8000D3F8606DC00603D421688868400705D534
:106D9000606D1021084360653574EBE7606DFF227C
:106DA0000132904302221043606588688207920F87
:106DB0005B48012A02D10A68D2072BD103236268FB
:106DC0009B079A4205D05B429A4202D05B009A42EE
:106DD00009D10A69920092080A6121680A69636808
:106DE0001A430A610CE00A69920092080A618168FC
:106DF0000F2292049143816081686268114381602F
:106E00002168CA6818239A43CA602168CA68A368BF
:106E10001A43CA60816801225206914381608168E9
:106E2000A28E52061143816020688168C90004D493
:106E3000816801221207114381602068C168394AC4
:106E40001140C1602069E168022825D0002001437B
:106E5000204620300278037B52035B001A43114323
:106E6000226B1143A26992031143E269D2031143D9
:106E70002268D3681943D160616A0A46FF3AC23A70
:106E800005D0A26A11432268D3681943D1604278C1
:106E90000121012A02D00BE00420D8E70078002865
:106EA00023D0606D202210436065A06D0843A0656B
:106EB000E06B012820681FD00169C90703D0016970
:106EC00049084900016120684169C908C900416158
:106ED00020684169A26B11434161A565606D80081E
:106EE0008000401C6065002070BD2068C2680123DE
:106EF0001B041A43C260DBE70269FF239B009A432D
:106F0000026120680269236CA66C1A43636C3343E8
:106F10001A430261206802690A430261D3E7000054
:106F2000002701401902FEFF10B586B00446142167
:106F30006846FEF74EFA0E492068884216D10D4881
:106F4000416B421511434163C16A01221143C16281
:106F5000C06A69461040059002200090032001900D
:106F6000002002900520000700F054FA06B010BD82
:106F70000024014000100240F8B50446406925464F
:106F800040350E4608280BD02068C068C00709D0DD
:106F9000606D202108436065002028740120F8BD41
:106FA000082700E00C2700F021FB009015E0701C82
:106FB00013D0002E05D000F019FB0099401AB04202
:106FC0000BD920680068384207D1606D042108435E
:106FD0006065002028740320F8BD206800683842EE
:106FE000E5D0606D01214902084360652068C168F1
:106FF00009058A0F0C21002A1BD12022125D002ACC
:1070000017D10268120714D5826853070122002B9A
:1070100008DB43688B434360606D13029843104361
:10702000606506E0606D202318436065A06D104325
:10703000A065A069002801D1206801600020F8BD8A
:1070400070B50446216800208968490721D4254687
:107050004035297C01291CD001212974E1690129CD
:1070600004D02046FFF784FA002811D1616D0A4A46
:107070001140FF220132114361650021A16529748D
:1070800022681C21116021688A6804231A438A60DF
:1070900070BD022070BD0000FEF1FFFF30B501465B
:1070A00020314A790023022A04D00422C2630B71E2
:1070B000012030BD026814680E25AC4314600268DC
:1070C0001468640864001460446C1C22144001229B
:1070D0001546006CA54045604A7118460B7130BDDD
:1070E00070B50024014620314A79022A03D00421D8
:1070F000C163012418E0026813680E25AB431360D6
:10710000026813685B085B001360436C1C22134029
:10711000012215469D40036C5D604A7100220A7190
:10712000816B002900D08847204670BDF0B4016C07
:107130000D6801680C68466C1C2304221E4017462B
:10714000B7402F420ED067070CD50C68A40602D4B6
:107150000C6894430C60416C19408A40016C4A6091
:10716000016B1AE00227B74002462F402032002F61
:1071700017D0A70715D50C68A40605D40C680A25F6
:10718000AC430C6001215171446C02211C40036C22
:10719000A140596000211171C16A002918D0F0BCCA
:1071A00008470827B7402F4212D0240710D50C6893
:1071B0000E25AC430C60446C01211C400B46A340DF
:1071C000046C6360C163517100211171416BE4E78C
:1071D000F0BC704770B504003CD01F4825681421EE
:1071E0002818FEF7F8F8800060641C48206402212B
:1071F000204620300246417129681948E368014061
:10720000A06866691843236933431843A369184388
:10721000E3691843236A1843084328600121A068E2
:107220008903884210D00D488030836A656C1C2128
:107230000D400F26AE40B3438362656C63680D401A
:10724000816AAB400B4383620020E06301215171EE
:10725000107170BD012070BDF8FFFDBF000002403D
:107260000F80FFFFF8B504468C46203001790025D9
:10727000012909D00126067141790027012905D08D
:10728000077102252846F8BD0220F8BD0221417190
:10729000E7632068016849084900016061462046AB
:1072A000FFF7F0F9206B00282068016801D00E225A
:1072B00005E0042291430160206801680A2211431D
:1072C00001602068016831430160DBE7F8B51A4EC0
:1072D0000546307C0F46012807D00120307417483E
:1072E000FFF7E2FA010002D021E00220F8BD002001
:1072F000C04338606C6814E02046FFF753FA0F482B
:10730000FFF7D2FA01460E48426808239A434260CA
:10731000426843159A434260002901D03C6006E070
:107320008034A8686A68C0018018A042E4D80020B0
:1073300030740846F8BD00009417002050C30000C8
:107340000020024005484168022211434160416823
:1073500001221143416000207047000000200240DC
:10736000F8B50C4C1646207C0F46012808D00120A9
:1073700020740948FFF798FA0025002802D006E09B
:107380000220F8BD65613E600348FFF78DFA257461
:10739000F8BD00009417002050C300001148416858
:1073A000C9070BD0EFF3108172B60F4AC2600F4AC3
:1073B000C26081F310884168C9070ED1416889070E
:1073C0000DD5EFF3108172B6094A0261094A0261D4
:1073D00081F310884068800701D5012070470020A4
:1073E0007047000000200240EFCDAB890504030286
:1073F000BFAE9D8C161514137047000010B50449DC
:107400004A69024202D04861FFF7F6FF10BD000052
:1074100000040140F8B5002303240125BDE03246F5
:107420002E469E40B446324079D00E79B607B60F4C
:10743000012E01D0022E17D186682746B6465E007F
:10744000B74000967646BE43B646CF68009EB7402A
:1074500076463743876046686746BE430F79FF0626
:10746000FF0F9F40374347600E79F643B6070ED0B3
:10747000C6682746B4465E00B646B7406646BE4379
:10748000B4468F687646B74066463743C7600E7984
:10749000B607B60F022E14D1DE08B60036180096D5
:1074A000366A5F07B446FE0E0F27B646B7406646FB
:1074B000BE43B4460F697646B74066463743009EE2
:1074C000376206682746B4465E00B646B740664651
:1074D000BE430F79B446BF07BF0F7646B740664636
:1074E000374307604E68B603B60F55D02E4F7E6BFC
:1074F0002E437E639F082D4EBF00BE190096B668CE
:107500000F27B4469E07360FB646B7406646BE43C1
:1075100005273F07B446B84202D1002715E03BE0FB
:10752000234FB84201D101270FE0224FB84201D1C9
:1075300002270AE0204FB84201D1032705E01F4F80
:10754000B84201D1052700E006277646B7406646D7
:107550003743009EB7601A4E36684F689643FF0364
:1075600000D51643164F3E607E684F689643BF03B2
:1075700000D51643124F7E60BE684F689643FF02E7
:1075800000D516430E4FBE60FE684F689643BF029B
:1075900000D516430A4AD6605B1C0A681646DA40D4
:1075A00000D03CE7F8BD00000010024000000140A0
:1075B0000004005000080050000C0050001C005057
:1075C000000401400069084000D001207047426972
:1075D00013460B401B0491430B4383617047002A01
:1075E00001D0816170478162704700000148806866
:1075F0007047000060010020024881680278891805
:10760000816070476001002010B5084800240168BF
:10761000402211430160204600F00AF8002801D002
:10762000012401E000F040FA204610BD0020024095
:1076300070B504460D4D7D202978C000FDF7CBFEC6
:1076400001460B480068FDF7C6FE00F029FF002840
:1076500009D1042C07D200222146401E00F04CFA2A
:1076600000206C6070BD012070BD00006001002032
:107670006C01002070477047F8B502F0BDFF594C0F
:1076800001252571208AFEF72DFE01467F20C005C9
:10769000FEF734FD544E316804F048FD3060FEF7CB
:1076A0009FFF607800280CD102215048FFF78AFF25
:1076B00002004F494F4818D00022FFF790FF0020EA
:1076C000E06202214948FFF77DFF4B4E002854D06D
:1076D0000020E062B08AFEF705FE434F396804F0EF
:1076E0006BFD5DD2454805705DE00122D103414844
:1076F000FFF775FF208AFEF7F5FD01467F20C005E4
:10770000FEF7FCFCE16A04F011FD3D49E0628842AD
:10771000D7DD39480127F926403000900A2130464C
:10772000FDF759FE002903D131493248FFF724F90A
:1077300002212E48FFF746FF002801D0002701E074
:10774000002F11D102212948FFF73CFF00280BD15F
:1077500004F020FC0098858004F07AFC642003F09B
:107760000BFF29492748C8600A2003F005FF30466F
:10777000761EF6B20028D1D1A3E7208AFEF7B2FD2B
:1077800001467F20C005FEF7B9FCE16A04F0CEFC9B
:107790001E49E06288429DDB1B491A48C86099E790
:1077A000164900200870708F401EFEF793FD39685F
:1077B00004F002FD05D86079002802D01448057055
:1077C00002E0134900200870708FFEF78BFD3968C6
:1077D00004F0F2FC04D26079002801D004F09CFB94
:1077E000F8BD0000240100205C01002000040050CE
:1077F00000800000000000509C0D00205E00002072
:10780000000040400400FA0500ED00E00000A04048
:107810006E000020704770B5040010D0022025468D
:107820002035A873204601F019FDA87B032805D058
:10783000204600F0C5F80020A873687370BD0120D1
:1078400070BD7047704710B5044600680168C943B1
:10785000C90708D18168C943C90704D10121416022
:107860002046FFF709FF20680168C943890708D44B
:107870008168C943890704D4022141602046FFF78B
:10788000F9FE20680168C943490708D48168C943E3
:10789000490704D404214160204600F003F9206820
:1078A0000168C943090708D48168C943090704D49A
:1078B000082141602046FFF7ADFF20680168C943F9
:1078C000C90608D48168C943C90604D4102141609F
:1078D0002046FFF7D0FE20680168C943890608D416
:1078E0008168C943890604D4202141602046FFF7FE
:1078F000A9FF20680168C943490608D48168C943C3
:10790000490604D4402141602046FFF79AFF10BD8C
:10791000F8B5040005D025462035A87B002802D004
:1079200006E00120F8BD00206873204600F05AF8F8
:107930000220A8732068C26884466368012B04D0C3
:107940000120A16AC005814201D11E20824319484D
:107950006169814201D0184802401848A668024077
:1079600018463043676A266A3E433043A66A30436E
:107970001043002B18D0012B03D00122D2059642D0
:1079800003D12369E2681A4310430A4A914205D0A1
:10799000A2691143E2690243084610436146C86088
:1079A0000120A8730020F8BD2369E2691A4310433F
:1079B000E3E70000FFFF00003F1FFFFFFEF119FF9C
:1079C00010B500680549884207D10548816B490018
:1079D000490881630D2000F073F810BD007C004061
:1079E0000010024010B50068084988420CD10848D0
:1079F000816BC20411438163002201210D2000F03C
:107A00007BF80D2000F06CF810BD0000007C0040F9
:107A1000001002400068C06970470000F8B50446D5
:107A20000220254620351746A8731D480268C30466
:107A30001A4302602068C2689B121A43C260206821
:107A400002690126324302612268102050602068DA
:107A500081611021204601F071FC03281FD02168AC
:107A600008204860206847610821204601F066FC34
:107A7000032814D0204601F0F1FBA87B03280ED088
:107A80002068816831438160206801693143016168
:107A900020680169042211430161AE730020F8BD22
:107AA00000040140704700000448416B012211436B
:107AB0004163816B020411438163704700100240EF
:107AC000002809DBC106C90E01208840034908606F
:107AD000BFF34F8FBFF36F8F7047000080E100E06E
:107AE000002805DBC106C90E012088400149086055
:107AF0007047000000E100E010B503F0E1FB10BDAD
:107B000002494A6882434A607047000000700040A2
:107B100002480168821511430160704700700040FF
:107B200002494A6802434A60704700000070004002
:107B300005480168022211430160044801690422DA
:107B40001143016130BF70470070004000ED00E05C
:107B5000F0B5154A1368154D54152D6A2340ED07ED
:107B6000ED0F002B04D0002D02D01668A64316603E
:107B70001668B608B600064316600D480769042665
:107B80003743076101290DD040BF20BF20BF0169E5
:107B9000B1430161002B04D0002D02D010682043B6
:107BA0001060F0BD30BFF2E70070004000000140FF
:107BB00000ED00E0F8B5044600780027534D80063C
:107BC00071D5524E403EB06BC00004D4B06BA905D5
:107BD0000843B06301274E480168C90511D4016804
:107BE000821511430160FFF701FD009005E0FFF7EA
:107BF000FDFC0099401A642837D845480068C00544
:107C0000F5D532680321090560680A4001409142B8
:107C100008D08103890F032904D13168890301D574
:107C20000120F8BD2A69032109040A4022D0084036
:107C300090421FD0207880061CD528692A69884385
:107C40000121C9040A432A612A698A432A612861F9
:107C5000C0050FD5FFF7CAFC009008E0FFF7C6FC8F
:107C60000099411A2B48814201D90320F8BD2869A7
:107C70008005F3D561688803800F032805D1326839
:107C80000005824301400A4332602869032261688B
:107C90001204114008432861002F04D0B16B012069
:107CA00000078143B1632078C00705D0E868A16868
:107CB000800880000843E8602078800705D5E868E0
:107CC0000C218843E1680843E8602078400706D526
:107CD000E86803218902884321690843E860207825
:107CE000000706D5E8680321090388436169084352
:107CF000E8602078000606D5E868032189048843F7
:107D0000A1690843E8600020F8BD0000401002406F
:107D10000070004088130000F8B50E46050038D00A
:107D20005E480068C007C00FB04214D25B4C2068A8
:107D30004008400030432060FFF758FC074605E04C
:107D4000FFF754FCC11B564881427AD82068C0070F
:107D5000C00FB042F4D12878524C800705D5E068B6
:107D6000F0218843A9680843E0602878C00752D012
:107D70006868022806D0032807D0216801280AD0A5
:107D8000890504E02168890301E02168890100294F
:107D900003DB0120F8BD4907F9E7E168890889009C
:107DA0000143E160FFF722FC0746686802280AD019
:107DB000032814D001281ED029E0FFF717FCC11BAF
:107DC000374881423DD8E0680007800F0228F4D18F
:107DD00021E0FFF70BFCC11B3148814231D8E0683C
:107DE0000007800F0328F4D115E0FFF7FFFBC11B4C
:107DF0002B48814225D8E0680007800F0128F4D184
:107E000009E0FFF7F3FBC11B2548814219D8E06860
:107E10000007800FF5D121480168C907C90FB14299
:107E200017D901684908490031430160FFF7DEFBBB
:107E3000074608E005E0FFF7D9FBC11B184881425F
:107E400001D90320F8BD15480068C007C00FB04233
:107E5000F1D12878400706D5E06807210902884358
:107E6000E9680843E0602878000707D5E068072143
:107E7000C90288432969C9000843E06000F03AF864
:107E8000E168094A0906090F515CC84007490860C2
:107E900007480068FFF7CCFBF8BD00000020024057
:107EA00088130000001002407EC300086C0100200F
:107EB00064010020044805490068C968044A49056E
:107EC000490F515CC84070476C010020001002400F
:107ED00097C30008044805490068C968044A890432
:107EE000490F515CC84070476C01002000100240EF
:107EF00097C3000870B51A4AD3681A490C20184075
:107F00008D0004280CD04E00082810D00C2810D06A
:107F100050680004410F0120C003491C884070BD17
:107F20001068C00601D5084670BD284670BD3046B1
:107F300070BD98020C4C000F205C1B029C0FD36894
:107F4000641CDB0301D5314603E01268D20600D47D
:107F5000294603F08FF922460023FDF72DF970BD65
:107F60000010024000093D008EC30008FEB5050068
:107F70007ED0FE4CE7680C20E66807400120000434
:107F800006402878C00747D0082F05D00C2F0AD10B
:107F900001200004864206D1206880033CD5686831
:107FA0000028E5D038E0012069680004814203D14F
:107FB00021680143216011E0052301221B04920482
:107FC0009942216802D111432160F1E78143216088
:107FD0002168014000912068904320606868002873
:107FE0000DD0FFF703FB009005E0FFF7FFFA0099C3
:107FF000401A64287BD820688003F6D50CE0FFF790
:10800000F5FA009005E0FFF7F1FA0099401A6428AC
:10801000F0D820688003F6D42878800756D5092345
:10802000E868042F0DD00C2F01D1002E09D00028B4
:108030003CD02168994301432160FFF7D7FA0646F7
:1080400028E02168490701D5002891D061681F22E6
:10805000120291432A691202114361602168994317
:1080600001432160FFF746FFE16809060A0F00E0BF
:108070008BE1BF49895CC840BE490860BE480068C2
:10808000FFF7D6FA002873D120E0FFF7AFFA801B84
:108090000228AFD820684007F7D560681F21090281
:1080A000884329690902084360600FE0206840089E
:1080B00040002060FFF79AFA064604E0FFF796FAC0
:1080C000801B022896D820684007F7D42878C0067D
:1080D00060D5002F0CD0A86900284AD02068FF2165
:1080E000013108432060FFF781FA06462EE0C1E027
:1080F0002068800502D5A8690028A6D060680721FD
:1081000049038843296A084360606068297F000248
:10811000000A090608436060286A410B0120C00379
:10812000491C8840E16809060A0F9149895CC840EA
:108130009049086090480068FFF77AFA002817D144
:1081400028E0FFF753FA801B0228A2D82068800598
:10815000F7D56068072149038843296A08436060AE
:108160006068297F0002000A09060843606011E088
:10817000E2E02168FF20013081432160FFF736FAF9
:10818000064604E0FFF732FA801B022872D8206806
:108190008005F7D42878794E000724D5686900282F
:1081A000306910D0012108433061FFF71FFA0090B9
:1081B00005E0FFF71BFA0099401A02285AD83069E7
:1081C0008007F6D50FE0400840003061FFF70EFA57
:1081D000009005E0FFF70AFA0099401A022849D8F2
:1081E00030698007F6D42878400766D500200290D1
:1081F000A06BC00006D4A06B012109070843A0634F
:10820000012002905E480168C90511D401688215F9
:1082100011430160FFF7EAF9009005E0FFF7E6F986
:108220000099401A642825D855480068C005F5D53E
:10823000FF20AA680130824203D1316901433161D4
:1082400011E001218902002A07D005231B029A426E
:1082500003D132690A433261EFE732698243326106
:10826000306988433061A868002810D0FFF7BEF954
:10827000009008E05FE0FFF7B9F901460098091A9D
:108280004048814257D830698005F4D50DE0FFF7AA
:10829000ADF9009006E0FFF7A9F90099411A3948B5
:1082A000814248D830698005F5D40298002804D06E
:1082B000A06B012109078843A063686A002866D083
:1082C0000C2F3ED0012636060228206805D0B04388
:1082D0002060FFF78BF905462FE0B0432060FFF7E1
:1082E00085F9074604E0FFF781F9C01B022822D870
:1082F00020688001F7D4E96AA86AE2680843296B1C
:10830000FD231B049A4311430843E0602068304377
:108310002060FFF76BF9054604E0FFF767F9401BA3
:10832000022808D820688001F7D530E0FFF75EF911
:10833000401B022801D90320FEBD20688001F5D42E
:1083400025E00128F8D0E06801210904AA6A01406B
:1083500091421AD10F218904EA6A0140914214D155
:10836000032189050840296B88420DE00010024076
:108370007EC300086C010020640100204010024010
:10838000007000408813000001D00120FEBD0020D5
:10839000FEBDF8B504000ED0FF27606A0537002542
:1083A00000280AD02561656126464036A562707CAA
:1083B000002807D00AE00120F8BD6068B842F3D079
:1083C000E561F1E73574204600F03EF80221717452
:1083D0002068026840239A4302602123A2686068F3
:1083E0009B021A4038401043E3688A021340184346
:1083F00023690B40217D1843C907C90F0843A169B0
:10840000931019400843E169382319400843216A51
:10841000802319400843A16A93001940084321684A
:108420000860A0690421000C0840616A102319400B
:108430000843216848602068C1699143C16165654E
:10844000012070740020F8BD10B586B004461421D8
:108450006846FCF7BEFF10492068884219D10F48D2
:10846000416B821411434163C16A01221143C1620D
:10847000C06A002110400590E02000900220019089
:108480000320039002910491052069460007FEF73E
:10849000C1FF06B010BD00000030014000100240D6
:1084A000094910B5401E884201D9012010BD074C72
:1084B00060610321081F02F003FF0020A061072074
:1084C0002061002010BD0000FFFFFF0000E000E081
:1084D000F0B502462032137E012B1ED00125157601
:1084E0000223537606687468B3687027BC430F682C
:1084F000274377600068AC07A04205D0084CA04233
:1085000002D0084CA04204D180244968A3431943F7
:108510008160557600201076F0BD0220F0BD00008D
:10852000000801400014014070B5050005D02C463C
:108530002034607E002802D006E0012070BD0020BB
:108540002076284600F010F802206076291D286861
:1085500002F0C8F80120A077A076E0762077607757
:108560006076002070BD000000680449884204D194
:108570000348416B042211434163704700080140E6
:1085800000100240F8B5054604462035287E002636
:10859000012817D00120287602206876226890688A
:1085A0007727FF23B8431B02984390600868502840
:1085B00038D00EDC20284FD006DC00284CD0102804
:1085C0001ED149E00220F8BD302845D0402817D1FF
:1085D0003AE060282ED0702819D001221203801AA8
:1085E0000FD090420CD1CB684A688968206802F0AD
:1085F000B2F820688168012292031143816000E093
:10860000012601206876002028763046F8BDCB6828
:108610004A688968206802F09EF8216888683843B3
:108620008860EEE7CA684968206802F00EF95021B8
:10863000206806E0CA684968206802F017F96021DE
:10864000206802F093F8DCE7CA684968206802F005
:10865000FCF840212068F4E7226801461046F0E764
:1086600010B586B0044614216846FCF7B2FE0D49E9
:108670002068884213D10C48C26A02210A43C262B0
:10868000C06A0191084005904803009000200290C4
:1086900003900620049069460448FEF7BBFE06B02E
:1086A00010BD00000008014000100240000400500E
:1086B000F8B5064604462036307E00270D460128D0
:1086C0000ED001203076002A0CD0042A1BD0082AB4
:1086D0002FD00C2A3ED00127002030763846F8BD36
:1086E0000220F8BD206802F049F82068816908225C
:1086F000114381612068826904218A438261206874
:108700008169EA6812E0206802F050F82068826906
:108710000121C9020A438261206881690122920213
:108720009143816120688169EA6812021143816185
:10873000D2E7206802F053F82068C169082211438B
:10874000C1612068C26904218A43C2612068C1698D
:10875000EA6812E0206802F05DF82068C169012231
:10876000D2021143C1612068C269012189028A4392
:10877000C2612068C169EA6812021143C161ABE7B6
:1087800070B5050005D02C462034607E002802D04C
:1087900006E0012070BD00202076284600F00FF88A
:1087A00002206076291D286801F09CFF0120A07737
:1087B000A076E076207760776076002070BD704705
:1087C00070B505462C4602202034002908D0042923
:1087D0000BD008290ED0627F012A10D0012070BD75
:1087E000A27E012AFAD1A0760AE0E27E012AF5D122
:1087F000E07605E0227F012AF0D1207700E0607763
:108800000122286801F09AFF0122286892070121BD
:10881000904205D0074A904202D0074A904204D1C4
:1088200082685207520F062A02D002680A43026089
:10883000002070BD000801400014014070B50446DE
:108840000D460068002201F079FF2068016A0C4A99
:10885000114203D101684908490001600120203418
:10886000002D06D0042D06D0082D06D060770020FC
:1088700070BDA076FBE7E076F9E72077F7E7000028
:10888000111100007047704770470000F8B502688A
:108890000446D06911689668A24B05461D40202306
:1088A000002D75D0F707A04DFF0FBC460D402F439C
:1088B0006DD02546C7078035002F06D0CF0504D5DB
:1088C000012717622A683A432A60820708D5F2070F
:1088D00006D0276802223A622A6804273A432A60AF
:1088E000420708D5F20706D02668042232622A68B9
:1088F000022632432A6002070AD50A461A40664613
:10890000324305D02668082232622E6816432E6054
:10891000020508D54A0106D501222668D202326234
:108920002A681A432A602A68002A39D0800606D5A8
:10893000880604D5616E002901D020468847286842
:1089400021688968490602D4282108422DD0204692
:1089500002F0B3F921688868400622D5EFF3108051
:10896000012282F310888B68402293438B6080F34E
:108970001088206F002814D06C498163206FFEF7A7
:10898000AFFB00280CD0206F816B08E000E012E004
:10899000850610D58D060ED5616EA9E02046884764
:1089A000F8BD2046FFF770FFF8BD2046FFF76CFFCB
:1089B00000202860F8BD256E012D7CD1C5067AD532
:1089C000CD0678D5102616622268906825464006A6
:1089D0004035002846DA216F086840680004000C22
:1089E000E8D02F8B8742E5D9688308680068800645
:1089F00033D4EFF31080012181F31088116837011F
:108A0000B943116080F31088EFF31080012181F3E6
:108A1000108821688A68520852008A6080F31088A2
:108A2000EFF31080012181F3108821688A684027C4
:108A3000BA438A6080F31088E36700202066EFF372
:108A40001080012181F3108821680A68B2430A600E
:108A500080F31088206FFEF721FB288B698B401A6A
:108A600081B231E0288B698B401A81B2688B002873
:108A7000A0D000299ED0EFF31080012585F3108847
:108A80001568FF272137BD43156080F31088EFF389
:108A90001080012282F31088226895686D086D00AD
:108AA000956080F31088E367002020666066EFF32E
:108AB0001080012200E00BE082F310882268136826
:108AC000B343136080F310882046FFF7DBFEF8BD48
:108AD000C50208D5750206D50120000510622046A2
:108AE000FFF7D1FEF8BD050606D50D0604D5A16E2B
:108AF000002900D052E7F8BD4006FCD54806FAD55B
:108B00002046EFF31081012484F310881468402577
:108B1000AC43146081F3108883670021816600F004
:108B2000E1F8F8BD0F08000020010004A9AB00081F
:108B300010B5040003D0A06F002802D007E0012088
:108B400010BD002174200155204600F027F8242094
:108B5000A06720680168490849000160204602F0CA
:108B60001DF90128ECD0606A002802D0204601F0EF
:108B700005FF206841680922D202914341602068C4
:108B800081682A2291438160206801680122114393
:108B90000160204601F058FF10BD0000F0B587B01D
:108BA000064614216846FCF714FC2C4930688842BC
:108BB00051D12B48416B0122920311434163C16A99
:108BC00001221143C162C06A0025104005900320B4
:108BD000400200900220032701A9A1C104200490B3
:108BE000052069460007FEF715FC1F4C1D48A560CF
:108BF000E56081C48027E560A76020202561606171
:108C00000002A0611848083CFEF7E4FA002801D0F1
:108C1000FDF7C6FD3467A662144C1248214614388D
:108C200020600320606010200831A1C16561A5614A
:108C3000E56120462562FEF7CDFA002801D0FDF758
:108C4000AFFDF466002201211B20A662FEF754FF4F
:108C50001B20FEF745FF07B0F0BD000000380140C3
:108C60000010024030000240041700204C17002082
:108C700070B5C36F202B2ED100290BD0002A09D04C
:108C8000012483682403A34206D10369002B03D186
:108C9000CB0701D0012070BD034660331C7D012C41
:108CA00019D001241C75002303660C4B04689C42F8
:108CB0000ED063681B020BD5EFF31083012585F3FB
:108CC000108825680126B6063543256083F3108891
:108CD00002F064F970BD022070BD00000048004041
:108CE000704770477047000001490248C160FDE7C6
:108CF0000400FA0500ED00E070B501240525E4024A
:108D00002D07002221462846FEF769FC0022042197
:108D10000948FEF764FC0A2002F035FC01222146D6
:108D20002846FEF75CFC0A2002F02DFC00222146BA
:108D30002846FEF754FC70BD00040050F0B585B025
:108D400014216846FCF745FB0420104F112402252E
:108D500000906946039501943846FEF75BFB019449
:108D60000524AE0224076946009603952046FEF7C7
:108D700051FB012231462046FEF731FC012204213D
:108D80003846FEF72CFC05B0F0BD00000004005092
:108D900070B501240525E4022D070022214628464E
:108DA000FEF71DFC012204210948FEF718FC0A20E9
:108DB00002F0E9FB012221462846FEF710FC0A20BA
:108DC00002F0E1FB002221462846FEF708FC70BDB8
:108DD00000040050F1B500240126F60205272546BF
:108DE0003F07002231463846FEF7F9FB0A2002F021
:108DF000CAFB012231463846FEF7F1FB6006040E3D
:108E000004210C48FEF7DEFB002801D0641CE4B20C
:108E1000052002F0B8FB6D1CEDB2082DE1D30098DF
:108E2000002803D0FFF768FF2046F8BDFFF7B0FF2A
:108E3000FAE7000000040050F8B5012605270546B2
:108E4000F6023F07002231463846FEF7C8FB0024F1
:108E5000E80901D0012200E0002204210E48FEF7BB
:108E6000BEFB6806050E0A2002F08DFB012231468A
:108E70003846FEF7B4FB0A2002F085FB002231469B
:108E80003846FEF7ACFB0A2002F07DFB641CE4B21E
:108E9000082CDDD3F8BD00000004005070B50E4C66
:108EA000012204212046FEF79AFB01220526D50265
:108EB000360729463046FEF792FB00220421204661
:108EC000FEF78DFB0A2002F05EFB002229463046A9
:108ED000FEF785FB70BD00000004005070B5012452
:108EE0000525E4022D07002221462846FEF777FBE0
:108EF0000B4E002204213046FEF771FB0A2002F0DF
:108F000042FB012221462846FEF769FB012204218B
:108F10003046FEF764FB0A2002F035FB70BD00000E
:108F200000040050F8B5154D002401220421284604
:108F3000FEF755FB062002F026FB01220527D6028C
:108F40003F0731463846FEF74AFB062002F01BFB7E
:108F500007E0641CE4B2FA2C03D9FFF7BFFF01203D
:108F6000F8BD04212846FEF72DFB0028F1D1002290
:108F700031463846FEF733FB0020F8BD00040050B0
:108F8000F8B501F093FD01F0C3FD3A480068C069EF
:108F9000FDF7C8FD384D394E287040213046FEF7A8
:108FA00011FB77010024002827D035480460E879B8
:108FB000002803D10120E87102F0C4F88021304676
:108FC000FEF700FB002806D0002208213046FEF7FD
:108FD00006FB012205E0012208213046FEF7FFFAD8
:108FE0000022052039460007FEF7F9FA254D264EE6
:108FF000A88C264F012803D019E0EC710022EBE782
:1090000023486946088072B680212248FDF7E0FBBC
:10901000002804D0022269461E48FDF77DFC62B696
:10902000AC8403F015F8642002F0A6FAFE60688CA8
:10903000012809D113486C844038048003F008F8F3
:10904000642002F099FAFE60288C012806D12C8455
:1090500002F0FEFF642002F08FFAFE6009480E4A1B
:1090600040380188914202D1C088002800D1FE60BA
:10907000F8BD0000801600202401002000040050EC
:109080005C010020DC0D00200400FA0500ED00E08A
:10909000AAAA0000384A0008AA55000038B50024E2
:1090A0006946202000F0ACF868460078572800D0C8
:1090B00001246946212000F0A3F8684600780328BF
:1090C00000D001246946222000F09AF86846007812
:1090D000402800D001246946232000F091F868461A
:1090E0000078082800D001246946302000F088F874
:1090F00068460078AA2800D001246946322000F092
:109100007FF80C486946008F0978884200D0012416
:109110006946332000F074F80648694640304088BC
:109120000978884201D1002C02D004490248C86065
:1091300038BD00009C0D00200400FA0500ED00E0A1
:1091400038B5FFF7FBFD5721202000F07AF8032106
:10915000212000F076F84021222000F072F808214A
:10916000232000F06EF8AA21302000F06AF81048A1
:10917000018F142901D8002901D1012101870C4C4C
:1091800040346188142901D8002901D1022161806D
:10919000008FC1B2322000F054F8A178332000F0E3
:1091A00050F8684600F006F80A2002F0ECF938BDE5
:1091B0009C0D002010B501460F2000F021F800287A
:1091C00000D0012010BD10B50446FFF767FE322025
:1091D000FFF732FEFFF7A6FEE0B2FFF72DFEFFF726
:1091E000A1FEFFF75BFE3320FFF726FEFFF79AFE96
:1091F0000020FFF7EFFD0446FFF770FE204610BD8C
:1092000010B50C46FFF7DFFF2070012010BD70B5D0
:109210000D460446FFF742FE3220FFF70DFEFFF732
:1092200081FEE0B2FFF708FEFFF77CFE2846FFF75D
:1092300003FEFFF777FEFFF751FE0A2002F0A3F9C5
:1092400070BD10B5FFF7E3FF012010BD10B5024857
:10925000FEF7F9FA10BD0000B8150020FEB504466F
:10926000002772B6334A01688B1804D13248C768A8
:1092700003208004074088680190C868009048690E
:109280008E69002B08D12C4940398B6ACD042B43C1
:109290008B628B6AAB438B62014631433CD02549DC
:1092A0002368CB4205D12449CA6803239B049A430F
:1092B000CA6025462035002810D021680A6901239C
:1092C0001A430A61216848610821204600F036F8F7
:1092D000032800D1A873216808204860002E10D010
:1092E0002068016901221143016120688661102113
:1092F000204600F023F8032800D1A873216810202D
:1093000048600C482168C14206D10B48C16803225D
:10931000920491433943C1602068016949084900BA
:10932000016121680198886021680098C86062B670
:10933000FEBD00000084FFBF4010024070B506462D
:109340000B480D46002409490068FCF744F87D21CC
:10935000C90048433168401E00D103240B682A46E7
:109360009A4301D00028F6D1204670BD204E00005F
:109370006C0100201CB5002116480091144A01918F
:109380000260C1631205426081600722826301228C
:1093900002610246C16020321170FF235170C23356
:1093A00043628162117301638161042241634261FE
:1093B000C161FDF7D5FC0848009080130190694613
:1093C0000448FDF77DFC00210248FDF71FFC1CBD91
:1093D000002401405C1500200200000408B5084884
:1093E000016B012211430163006B012110400090C9
:1093F00000220A20FEF780FB0A20FEF771FB08BD61
:1094000000100240F0B587B014216846FBF7E1FF79
:109410004A48C26A04210A43C262C26A0A400592EB
:10942000C16A80273943C162C16A39400591C16A66
:1094300001252943C162C16A29400591C16A0226FA
:109440003143C162C06A81213040059005202A461F
:1094500009010007FEF7C3F8012239493948FEF730
:10946000BEF8002238493748FEF7B9F891210520A7
:10947000002209020007FEF7B2F811200004019053
:10948000002405206946009502940007FDF7C2FFFD
:10949000102000900520694603960195029400076C
:1094A000FDF7B8FF05200090112001900294694655
:1094B00003942448FDF7AEFF212000040190694683
:1094C000009602951F48FDF7A5FF204800900294E2
:1094D0006946019503941B48FDF79CFF912000020B
:1094E0000090052002946946019503940007FDF75A
:1094F00091FFE80200901120019005200294694636
:1095000003940007FDF786FF402000900194694610
:1095100002940C48FDF77EFF69460A4800970295C1
:109520000194FDF777FF002201210520FEF7E4FA00
:109530000520FEF7D5FA07B0F0BD0000001002408C
:10954000050200000004005008300000083200004E
:1095500010B50F4C0D482060FF20053060600020E2
:10956000A060E06020616061E06101212062490249
:109570006062A161A0620720E0622046FEF709FF59
:109580002068016840221143016010BD0030014095
:10959000E815002010B58AB00024049405940694C0
:1095A0000794089419480994009401940294164968
:1095B000039401600921846041600461144944619D
:1095C000C160FEF7B1FF01200003049004A90F4819
:1095D000FEF7D8FF0D48FFF7D3F8089408A90B4809
:1095E0000994FEF775FF602000900A4801900294EC
:1095F0000422694603940548FFF75AF80348FFF729
:109600002FF80AB010BD00000008014040160020ED
:10961000930400004902000000B585B0142168469B
:10962000FBF7D7FE0E480D490160E1214902416078
:1096300000218160C160016181610C22C1614261D0
:109640000162302141620121090381634900C16344
:10965000FFF76EFA01F070FD05B000BD0038014063
:109660008016002070470000F0B589B00A2002F093
:1096700073FA7D20400102F089FAFF4C0025A570A5
:10968000FE482066607C0C2801D30B206074607952
:109690000A2801D90A206071F948E570F94E00786E
:1096A0003071F949A079097840000843A17D89000B
:1096B0000843F071E06BF070010A3172401CE06306
:1096C0006079B07442003046F0491330FBF722FE57
:1096D0006079EE4982004000801960311330121D1C
:1096E000FBF718FE60790621420048438019E849DB
:1096F0001730921CFBF70EFE2E20205E002803D0B0
:10970000E449098A0818E0856079DB49C000223104
:1097100082190B7B53764B7B937606227272DE4A5C
:109720001D301278B272A28C3273D64A0B79133A7A
:109730001375497951750022D24902F0F7FA607920
:109740000021C0001D3002F003FBD448FEF762F98F
:1097500001272085BF0309E0D048FEF75BF980B2FE
:109760002085E18EFF392D39884206DB81B2E08EFB
:109770008142F1D3C0198142EED8022002F03CFAB6
:10978000C0480126C571A574A5732674E573C34846
:10979000FEF740F960850746E5706079FCF75DFBF0
:1097A000BF4AC04BFCF75CFB01F082FE0022BE4BBF
:1097B000FCF77CF8FCF704FB0006C00CC01980B273
:1097C000F103A085884201D3401AA085B748E06420
:1097D0002079401C2071B148FEF71CF92085AB4868
:1097E000A54F643840370690B1E1AC48FEF712F956
:1097F00020850BE0A948FEF70DF980B22085A18DE8
:10980000884203D3AA4A8918884207D300210F202F
:1098100002F022F9A74920640842EBD0206C411CD9
:109820001FD040047ED58122D20100210F2002F0FA
:1098300052FA0021102002F00FF941069348490E18
:1098400000227C38E16502F03DF9002002F09EF92B
:10985000002002F050F98D487C38417A0729C3D1A5
:1098600001E001F04FFD02229349401DFBF725FD69
:109870000028B9D102F0B0FAE167A06702F099FAC6
:109880007D4B803303C3E0788049401CE07083390E
:109890000B7A68460370497A417000880390E18C26
:1098A00088427DD1774985488C31C98E01807548C1
:1098B00071498C30008F48847848FEF7ABF82085DA
:1098C00001F0DCFF6C48FF228030016840685204E0
:1098D0000023891858410206080A1043410849002C
:1098E00000900A0E080264498031CA6088606548A9
:1098F000E36F0A30A26F02F051FA6079810061488B
:1099000008185D49163080310CC902F047FA5A48F0
:109910008030C36882685B48123002F03FFA082149
:10992000584800E006E14172B430C07C000960751F
:1099300014D05648022260497738FBF7BEFC002855
:109940000CD15048A674C671E06D50491638C2B2A9
:109950006639C81DE274FB30FBF7DCFC607900223D
:10996000800048491C3002F0E1F960790021800054
:109970001C3002F0EDF9009802F0E7F8012002F047
:109980003BF9207302214E48FDF71CFE00281DD034
:1099900000213D4801703B498C31488E049000E025
:1099A0005AE03881888E78818446A06CFF31053179
:1099B000E0640860DC392065C97C0907090F0329C8
:1099C00000D02175E16D1C2902D015E00121E0E7EE
:1099D0002C49294A8C31C98F1186069B2C4A1B8839
:1099E0001380884207DD002805DD002903D0207E92
:1099F000401C207600E025762571A6730498B88176
:109A00006046F881E673608C2E49FF30C33080B227
:109A1000608488420CD949424018608427487D22DE
:109A20000188D200491C89B20180914200D305808F
:109A300022487D210088C9004843618C4018606538
:109A400000F076FD207B002805D100210F2002F0D8
:109A500003F80006F9D583E0FCF77AFF0B4A0321EF
:109A60009032115407498C314A8E3A81898E79811E
:109A7000E26D1C2A2ED127E0580000203F420F0043
:109A80002401002010120020580100204013002063
:109A90007C140020DC0D002034010020B8150020CB
:109AA000B81E85EB51B8CE3F00000840A0860100EB
:109AB000983A000000D027244801002054010020DB
:109AC00000040050E7030000624B4200D318069ADE
:109AD00012885A808000604B5F4AD43B02905E49F6
:109AE00082189B8F138030314118A26C4A605B4909
:109AF00040185B4916300CC902F050F9216EA06C79
:109B0000884207DA544A02995158012902D1206645
:109B1000039905915049029A8958814217DD01291C
:109B200015DD2146002812DD0398C8840220087044
:109B300065730CE04B4A00210F2002F0CCF86079ED
:109B4000E178401C814202D0002001F0D4FF208D3A
:109B5000A18D884200D248E6434A89188842FAD843
:109B6000A07B012801D00220A07301F087FE3D4AAE
:109B700000210F2002F0AFF82179002917D03B48CF
:109B80000288900013188B4200D22570002000F04C
:109B9000E9F8A07C00283BD02F496C310B78A372E8
:109BA000487860728A782272022B17D030E0E16C1C
:109BB000226E323920468A420EDAC1792B4A491C7C
:109BC000C9B2C171128852008A42E2D20599C18499
:109BD000022101706573DCE7E571DAE710280ED029
:109BE000C82815D2224BC91C1D60224B1818FBF740
:109BF00091FB02F02DFA642001F0BEFC31E61E4D0F
:109C000028684000000E03D1C878FCF76BFB286081
:109C100000202378627B657910E00F4E0E4F4100E3
:109C2000303E183F765A7F5ABE4205D00A4F022373
:109C300000220126483F7E52401CC0B2A842ECD30D
:109C400023706273074A002180320F2002F043F82C
:109C500009B0F0BD7C140020701300201012002009
:109C6000D800002000D02724983A000034010020BA
:109C70005C0100209C0D00204C010020F8B52E4C0A
:109C80000546E06E2D4A281A411E2067914215D2E2
:109C90001A21615E081AFCF7D8F8294A294BFCF70B
:109CA000DFF8064632200F46205EFCF7CEF832463B
:109CB0003B46FBF7FBFDFCF74DF860860020607625
:109CC0001D481C23C35E828C1F48008884461F48A1
:109CD00006881DE06046484380181D4F80B23880DA
:109CE000302778436427643078431A4F6066C01980
:109CF00085420BD2C8B2184932220880606EA25E3B
:109D0000411BC9188918A166E066F8BD491C617637
:109D1000617EB142DED330204243104864211018E6
:109D200048430F494118E16660663221401B615E7D
:109D3000C0184018A066F8BD58000020CF070000EA
:109D40009A9999999999B93F4201002034010020CC
:109D50005601002078ECFFFF40010020742700002E
:109D6000C0BDF0FFFEB5294D2988491C8FB2284996
:109D70002F800E88FCF769F8264A274BFCF770F80D
:109D80000191009025483146FBF725FB244C218F9B
:109D90004218B74206D3002028802248019E10189E
:109DA000009D02E01046019E009DFCF756F83346E8
:109DB0002A46FBF77BFDFCF703F8A086012580B25D
:109DC000ED03A84201D3401BA086E08BFCF745F8C9
:109DD000154A164BFBF79AFD0646A08E0F460090DB
:109DE000FCF73BF832463B46FBF760FDFBF7E8FF2C
:109DF00080B2E086A84201D3401BE0860C4900985F
:109E00000968486100982087FEBD000040010020DD
:109E1000340100201904560E2D624040E17A000002
:109E2000580000201F050000F853E3A59B843E4026
:109E3000B815002070470000F0B589B000200490EC
:109E40000A2001F089FE7D20400101F09FFEB34809
:109E500000228270C16BB34C491CC163B049C38DF1
:109E6000098A2546C918C1852146C2751331079153
:109E7000473103916D393135AB4F22300591029056
:109E8000A64E0F21A948717100782071A84AB079B7
:109E9000127840001043B27D92001043E071B08F01
:109EA000E070000A2072A17431461E229C3107988E
:109EB000FBF730FA402228469E49FBF72BFA02991D
:109EC00003980A7BC274497B0175092060729A4825
:109ED0000078A072B08C2073F07D410030469C3039
:109EE000091805980A78027549784175762000228C
:109EF0008C4901F01BFF70790621484300211C307A
:109F000001F026FF022001F077FE00210F2001F072
:109F1000A3FD38423064F8D0306C411C18D04004A6
:109F20007ED58122D20100210F2001F0D4FE002134
:109F3000102001F091FD41067A48490E0022B4300C
:109F400001F0C0FD7748B430417A022902D0BDE06B
:109F500001F0D8F902227949401DFBF7AEF900283B
:109F6000F5D16E480222C07D41006C489C30091832
:109F70006C48B530FBF7A1F90028E8D101F02CFFBF
:109F8000664AD167906701F014FF644A803203C2C9
:109F9000049800282CD1012004906248684E8C302F
:109FA000C08E604930805D488C31098F418465489E
:109FB000FDF730FD5949644A0885488CFF30C330AD
:109FC00080B2488490420CD952428018488430882C
:109FD0005D4A401C80B20B323080904201D3002099
:109FE000308030887D22D20050434A8C80184865EA
:109FF0004C4869468C30428E0A80808E48804949A0
:10A000000422B531C81FFF38FBF784F94348494A99
:10A01000C07D0099800011504049803103C900E0A3
:10A0200075E0FF235B040022C01851410906060AAF
:10A030000E43304601F089FD710849000A0E0802FE
:10A04000364900268031CA6088603448C36F826F09
:10A050003448483801F0A2FE304880300CC83148FE
:10A06000443801F09BFE2D488030C36882682D483B
:10A07000403801F093FE2B49002252393C2001F078
:10A0800055FE00213C2001F063FE012001F0B4FDEB
:10A090002249087308468078401C887001210520F9
:10A0A000C9030007FCF768FC1C48007B002805D1A9
:10A0B00000210F2001F0D0FC0006F9D580220021FC
:10A0C0000F2001F008FE1548467002E013490120F8
:10A0D00048701248C17D491CC9B2C1750F2900D210
:10A0E000CEE60498002810D10C4A1849908C00281C
:10A0F00002D00B88984201D908889084144980B214
:10A100000988401E48431349088009B0F0BD124A2F
:10A1100000210F2001F0DFFDD8E7000058000020EB
:10A12000DC0D00201012002000D027242401002084
:10A13000580100202C140020340100204801002088
:10A1400054010020B8150020E70300003001002072
:10A150002E0100202C01002000902724F8B5314961
:10A160002F48086001F016FF2F4800F0A1F92F4C8E
:10A17000E0822D48801C00F09BF920832A48001DB6
:10A1800000F096F960832B4829494180014640310F
:10A190000979294F0906090E617006D1C78001218E
:10A1A000C1870A21418700218187244AC18E11700D
:10A1B000C18F6171818FA171817AE17085880521DC
:10A1C00065626181C6883046FBF705F9A0810146CA
:10A1D0002846FBF700F98800081885B21648258143
:10A1E0006843FBF73AFE164A164BFBF78FFBFBF76B
:10A1F000E7FDE081658231463846FBF7ECF82082C6
:10A200000146C820FBF7E7F8E0830120A083FCF7B4
:10A21000B7FBA082E2890C490C48FDF7FFFBF8BDB3
:10A2200065B1000850000020004F00082401002004
:10A23000310200009C0D0020E80300000000002017
:10A24000F853E3A59B843E40FF7F0000B815002033
:10A25000F8B5744C00202071734D01202880734E96
:10A26000C8203080E07A401CE072C00706D0A08C85
:10A27000411EA184022801D2C820A0840120C0432D
:10A28000FFF770FD0A2001F067FC7D20400101F01E
:10A290007DFC02216648FDF795F900287ED000205C
:10A2A000644980000978654F49000843624909788C
:10A2B0000843B872102078726148C1887D20C000C0
:10A2C000FBF789F878735F485D490078B8733846C2
:10A2D0000B308A780270C97841705949421C20318C
:10A2E0000B7ED370497E11715549D01C22310B7EF3
:10A2F0005371497E9171524940310A7C0271497C07
:10A30000417100223946172001F010FD002117206D
:10A3100001F01EFD022001F06FFC4B4F00210F20C9
:10A3200001F09AFB38422064F8D0206C411C77D0B1
:10A33000400471D58122D20100210F2001F0CBFC15
:10A340000021102001F088FB41063C48490E002204
:10A35000B430E16501F0B6FB384FB437787A112894
:10A360005AD102223949781DFAF7A7FF002853D1A4
:10A37000F81F027A69460A70407A4870B97A2980D3
:10A38000C820FBF728F83080387BA0843846304D51
:10A390002838C08E28802348394600E03EE028391E
:10A3A000098F41842B48FDF735FB2085608C2A49B5
:10A3B000FF30C33080B2608488420CD949424018D3
:10A3C000608428882449401C80B20B312880884250
:10A3D00001D30020288028887D21C9004843618C52
:10A3E0004018606500F0A4F868460088E0841349CE
:10A3F000B87CC7316071420008460D466930FAF7F3
:10A4000089FF6079294642001448FAF783FFA08C3F
:10A41000FF2801D003202070F8BD01E001203FE7B4
:10A4200000F070FF5800002034010020420100209D
:10A4300000040050290100202A01002010120020F1
:10A440009C0D00200000002000D02724480100209F
:10A4500054010020B8150020E70300005813002025
:10A4600070B586B014216846FAF7B3FF01250F4E88
:10A47000ED03002229463046FDF7B1F80120002403
:10A48000019002946946009503943046FCF7C2FFA0
:10A490000320019002946946009503943046FCF72E
:10A4A000B9FF022001F068F806B070BD000400504A
:10A4B0000088704770470000F8B5044600206A46DF
:10A4C0001080194D55222A70AA226A700322AA70A0
:10A4D000661DEE702A716971144A49008918AC71C1
:10A4E0002246E81DFAF716FF002007E029186A4601
:10A4F0008978128889186A461180401CB042F5DBC1
:10A50000611DA81CFCF7A4F80146684601802919C2
:10A510000078C871684640780872214609310248BF
:10A5200000F00AFCF8BD0000F61400209C0D00208D
:10A53000FEB5FFF7A3FB2548FDF76CFA244C86B265
:10A54000268560790A21081AC000FBF77EFC0746C1
:10A550000191A06EFBF781FC1E4A1F4BFBF7D6F959
:10A5600000900D463046FBF778FC2B46009AFBF72F
:10A570009DF93A46019BFBF799F9FBF721FC85B25F
:10A58000A586E08BFBF769FC124A134BFBF7BEF97B
:10A5900006460F462846FBF760FC32463B46FBF773
:10A5A00085F9FBF70DFC81B20120C003E1868142F1
:10A5B00001D3091AE186854201D3281AA0860349EE
:10A5C000A08E096848612087FEBD0000B8150020F4
:10A5D00058000020F853E3A59B843E40034A1168CD
:10A5E000382389B29943014311607047003001401C
:10A5F00010B5FDF701F810BD10B59AB034216846CA
:10A60000FAF7E7FE14210DA8FAF7E3FE1C2112A8C1
:10A61000FAF7DFFE1B4801680324E402A143C214D9
:10A6200089180160FDF774FA17480169A1430161B7
:10A6300006200090FF20013002900120039010209E
:10A6400004900220099040040B90000100240C901B
:10A650000A946846FDF78AFC0F200D9003200E90A7
:10A660000F941094012111940DA8FDF755FB812042
:10A670001290032080041890149412A8FDF79AFAFF
:10A680001AB010BD00700040401002401048016830
:10A69000821511430160C1680E4A1140C160016812
:10A6A0000D4A1140016081684908490081600168D4
:10A6B0000122920491430160C168FD22120491437A
:10A6C000C1600021016106490448886070470000AC
:10A6D000001002400C40FF88F6FFF6FE0050000814
:10A6E00000ED00E070B5026801239B07114C124D8C
:10A6F000984203D0A04201D0A84203D17026B243B1
:10A700004E683243984203D0A04201D0A84204D1FF
:10A7100003231B029A43CB681A4380239A430B6995
:10A720001A4302608A68C26209688162012141613C
:10A7300070BD0000000801400014014010B5CB06B8
:10A74000DB0E0121046A99408C430462016A9A403D
:10A750001143016210BD30B58468FF252D021B0234
:10A760001343AC430B432343836030BD82687023A3
:10A770009A430A4307210A438260704730B5026A50
:10A78000520852000262026A456883697024A3433A
:10A790009C080B68A40023430224A2438C684560F4
:10A7A0001443836149684163046230BD30B5026A75
:10A7B00010239A430262036A456882697324240263
:10A7C000A2430C6824021443202293438A68456004
:10A7D00012011A43846149688163026230BD30B559
:10A7E000026AFF2301339A430262026A4568C36921
:10A7F0007024A3439C080B68A40023430124640233
:10A80000A2438C68456024021443C3614968C16354
:10A81000046230BD30B5026A01231B039A43026211
:10A82000036A4568C26973242402A2430C682402A7
:10A8300014430122520393438A68456012031A436A
:10A84000C46149680164026230BD30B5036A046ABC
:10A850006408640004628469F025AC431201224359
:10A860000A24A3430B438261036230BD30B5036AFF
:10A870001024A34303628469036A0F252D03120386
:10A88000AC432243A024A34309011943826101621E
:10A8900030BD0000F8B5102405252D07AC62AF20AF
:10A8A000800000F070FEAC6101F0EAF82D4C2E4FF4
:10A8B0002E4E60670BE001F0E3F86067FEF760FB87
:10A8C000606C411C6164142801D92948C760606F1D
:10A8D000B042F0D10026666420780127FF03030010
:10A8E00000F0E0FC05040C192D303200012239463D
:10A8F0002846FCF774FEFFF7ABFC06E00122394660
:10A900002846FCF76CFEFFF797FA002239462846E6
:10A91000FCF765FE18E0607B0122401C607339463D
:10A920002846FCF75CFEFCF747F80022394628462B
:10A93000FCF755FE607B052806D9267004E0FEF77B
:10A9400093FE01E0FFF778FA02210A48FCF73AFE8D
:10A95000002805D000200849087000F077FFF8BDF6
:10A960000120F8E7580000200400FA053001CADE93
:10A9700000ED00E0000400505801002010B5818C6B
:10A98000C90707D001684A6801235B049A43836AB8
:10A990001A434A60818C890707D501684A680123F8
:10A9A0001B049A43C36A1A434A60818C490707D53E
:10A9B00001684A6801239B049A43036B1A434A6067
:10A9C000818C090707D501684A680123DB039A4394
:10A9D000436B1A434A60818CC90607D502689168A7
:10A9E00001231B039943836B19439160818C890672
:10A9F00007D501688A6801235B039A43C36B1A4336
:10AA00008A60818C490612D503685A6801210905BC
:10AA1000046C8A4322435A60026C8A4207D102685E
:10AA2000516803235B059943436C19435160818C42
:10AA3000090607D501684A680123DB04806C9A4344
:10AA400002434A6010BD0000F8B50446002680307D
:10AA50000660FCF7CBFD054620680068124F000732
:10AA600009D501212B46002249052046009700F018
:10AA7000EDFA00280DD12068006840070BD50121B0
:10AA80002B46002289052046009700F0DFFA0028B7
:10AA900001D00320F8BD2020A067E067266660345F
:10AAA00026750020F8BD0000FFFFFF01F8B5154C2A
:10AAB000C826E078002823D16079002820D1012021
:10AAC0006071114D686B0027002818D0686BC82191
:10AAD000081A0FE00D48E168405C61698847E0684A
:10AAE000401CE060E068C82800DBE760696BC820B4
:10AAF000401A761EE168814201D0002EEADC6771BF
:10AB0000F8BD00003C00002000000240D40C0020F2
:10AB100070B5224CE07800283FD1207900283CD144
:10AB2000012020711E4EF16900250906002933DA43
:10AB30002156625791420AD1F06940062CD5A0797E
:10AB4000002829D0A5712089401C208124E0A1790A
:10AB5000002903D1A0710A2000F015FD0020205625
:10AB6000CC2148430F494218206912181279B26269
:10AB7000401C00222061A256CC235A4389588142AE
:10AB80000ADC25612078401C207020780E2800D136
:10AB90002570A078401CA070257170BD3C0000207D
:10ABA00000380140AC01002010B5806A0022014647
:10ABB00040314A834A82FDF767FE10BD70B5846A52
:10ABC000A06FE56F2168896800260906002906DA6A
:10ABD000212804D152200653204600F09DF8206819
:10ABE0008068400606D5222D04D15A2006532046FF
:10ABF00000F063F8204680300168102211430160A4
:10AC00002046FDF741FE70BD10B501460968806A17
:10AC10000968890638D400225A210A52EFF31081BC
:10AC2000012282F3108802681368FF240134A343D1
:10AC3000136081F31088EFF31081012282F31088F2
:10AC4000026893685B085B00936081F31088EFF300
:10AC50001081012282F31088026893684024A34384
:10AC6000936081F310882021C167016E01290BD107
:10AC7000EFF31081012282F3108802681368102418
:10AC8000A343136081F31088016E012902D0FEF7FF
:10AC900027F810BD5821095AFDF7F4FD10BD10B575
:10ACA000806A016E012902D0FEF71BF810BD582101
:10ACB000095A4908FDF7E6FD10BD10B5EFF3108104
:10ACC000012282F3108802681368FF242134A34311
:10ACD000136081F31088EFF31081012282F3108852
:10ACE000026893685B085B00936081F31088016ED3
:10ACF00001290BD1EFF31081012282F31088026841
:10AD000013681024A343136081F310882021C167C6
:10AD100000210166416610BD10B5EFF310810122DC
:10AD200082F3108802681368C024A343136081F380
:10AD300010882021816710BD70B5164CE278002A7A
:10AD40000CD12279002A09D10122E2700025C829FC
:10AD500003DC0222A256002A01DCE57070BD01234B
:10AD6000E356CC2253430C4AD1500123E356CC2660
:10AD700073439B180A460146181DFAF7CBFA607810
:10AD8000401C607060780E2800D16570A078401E6D
:10AD9000A070E2E73C000020AC010020F8B50446BA
:10ADA000016880682369E6691843636900253343B5
:10ADB0001843724A0B68724E334003430B6021689C
:10ADC000486803231B039843E368184348602168DD
:10ADD000A069914201D0236A18438B680B26360282
:10ADE000B34303438B606749236867488B420CD1A8
:10ADF000C0688007800F06D0012839D0022835D0DE
:10AE0000032821D11EE001271FE060498B420AD1AF
:10AE1000C0680C21084027D0042829D0082825D054
:10AE20000C2811D10EE093420ED1C168032080029C
:10AE3000014019D001208002091A19D0091A15D031
:10AE4000814201D1082700E010274F49504840397E
:10AE50008600934232D1002F0CD0022F0DD0042F48
:10AE600010D0082F7FD126E00027EEE70227ECE77D
:10AE70000427EAE7FDF71EF806E00968C90605D4CD
:10AE8000304603E0FDF736F8002872D062685100C2
:10AE90005118814267D81103814264D3010E060222
:10AEA0005008002330185941FAF786F903210902A6
:10AEB000411A384A55E00120C003E7E70122E3695F
:10AEC000D20393422BD13B0000F0ECF90906090CA8
:10AED0004D114D4D4D274D00FCF7ECFF09E0FCF7FF
:10AEE000F9FF06E00968C90605D4304603E0FDF71E
:10AEF00001F800283DD0616840004A088018FAF740
:10AF00006AFA80B20146244A103991422BD8511C6A
:10AF100001400007400F084329E01046EBE73B00E3
:10AF200000F0C0F90906090C21122121212321007A
:10AF3000FCF7C0FF0AE0FCF7CDFF07E00968C9068F
:10AF400006D4304604E00EE0FCF7D4FF002810D011
:10AF500061684A081018FAF73EFA80B201460E4AB4
:10AF60001039914203D9012503E01046F0E721682A
:10AF7000C86000206066A0662846F8BD0048004012
:10AF8000F369FFEF003801404010024000440040E8
:10AF900000093D00FFFC0F00EFFF0000F8B504467C
:10AFA0004165403000262746028380373E602220DC
:10AFB000E0672546206F603500281BD02049C1621C
:10AFC000216F20480863216F1F484863206F134694
:10AFD0008663606D2168844662462431206FFCF7E9
:10AFE00041F9002806D0102038602E752020E06737
:10AFF0000120F8BD2E75EFF31080012181F3108838
:10B0000021680A68FF2301331A430A6080F310881D
:10B01000EFF31080012181F31088226893680B43BD
:10B02000936080F31088EFF3108081F3108821681B
:10B030008A6840231A438A6080F310880020F8BD94
:10B0400009AC00089FAC0008BDAB0008FFB581B09B
:10B0500005461746044660350A9E55E0701C53D0DD
:10B06000FCF7C4FA0499401AB04230D8002E2ED012
:10B0700020680168490747D5C069C043000543D42B
:10B0800001202168C0020862EFF31080012181F3E2
:10B09000108821680B68FF22A13293430B6080F374
:10B0A0001088EFF31080012181F3108821688A68ED
:10B0B000520852008A6080F310882020A067E06761
:10B0C0008034206000202875032005B0F0BDEFF328
:10B0D0001080012181F3108821680B68FF22A132C2
:10B0E00093430B6080F31088EFF31080012181F30C
:10B0F000108821688A68520852008A6080F310889C
:10B100002020A067E067DDE72068C16902988843D6
:10B1100004D00020B842A1D00020D6E70120F9E7F2
:10B1200010B504491020096808620248FDF7AEFB1B
:10B1300010BD00008016002001490D208870704766
:10B140003C00002010B5FEF749F9FEF765FAC82269
:10B1500002490348FDF78CFD10BD0000D40C00200F
:10B1600080160020F8B53E4C002321783D4A1D464C
:10B17000082910D0072947D0062950D0052952D0D8
:10B18000042953D0032954D0002956D0012958D07E
:10B1900002295AD05BE0A17800264A1F04E0314F13
:10B1A000BF5DFB189BB2761C9642F8DB6679277967
:10B1B0009A195118E3786278C9188918C919401882
:10B1C000C0430006000E1AD1012E14D0022E16D153
:10B1D00025482449C018FAF79DF800F039FF64208B
:10B1E00000F0CAF9BFF34F8F21492048C860BFF370
:10B1F0004F8F00BFFDE759081046FFF75DF9257036
:10B20000E570A570A571F8BDA1795054491CC8B26C
:10B21000A071A178491F8842F5D1082001E0607033
:10B2200007202070F8BDE0700620FAE76071052065
:10B23000F7E7A070E5700420F3E7552807D1012057
:10B24000EFE7AA2803D10220EBE7032803D02570FB
:10B25000E570A570F8BD032020702071F8BD0000D6
:10B260001C010020921400209C0D00200400FA050F
:10B2700000ED00E0F8B5040C8BB2264682B25E43C6
:10B280000D0C1046370C58433604801900217941C3
:10B2900016466E43370C36048019794126466E43B4
:10B2A0008919F8BD30B47446641E2578641CAB421D
:10B2B00000D21D46635D5B00E31830BC18470000F8
:10B2C0008307FF22DB0E9A408907090E9940002868
:10B2D00008DB830809489B001B1818689043084343
:10B2E000186070470007000F0838830804489B0067
:10B2F0001B18D86990430843D861704700E400E008
:10B3000000ED00E0BFF34F8F04490348C860BFF36E
:10B310004F8F00BFFDE700000400FA0500ED00E0DC
:10B3200008B50021684601706B46012202212C20DD
:10B3300000F0E0FC0221684601706B4601222C20DF
:10B3400000F0D8FC08BD000038B504466D20694601
:10B3500008706B46012207492E2000F0CBFC0649FD
:10B36000002C01D0054A00E0054A2E2000F0A8FC80
:10B3700038BD00000608000006180000070600009F
:10B380000716000038B504466B460222002136201D
:10B3900000F07CFBB3212300FFF784FF0E0F08159C
:10B3A0003A3A3A3A1C273A3A2F34483A002168464A
:10B3B000017040784108490014E069460878800827
:10B3C0008000401C04E06946087880088000801CEA
:10B3D00008701DE0684602780A40483202704178E1
:10B3E000802001436846417012E0684602780A40B6
:10B3F000027040784106490EF4E769464878022118
:10B40000084303E069464878FD21084069464870D2
:10B410006B4601220021362000F06CFC012200ABBB
:10B4200011463620013300F065FC38BD69460878C6
:10B43000CF21084069462030CAE708B50321684695
:10B440004170012101706B4602220021362000F07C
:10B4500051FC0122D20306212D2000F031FC0120F5
:10B4600000F08AF80120FFF78DFF08BD08B5020A39
:10B4700069464A7008706B46022204212D2000F0B4
:10B4800039FC0320694608706B46012206212D20F5
:10B4900000F030FC0020694608706B46012206214E
:10B4A0002D2000F027FC0A212D2000F0D5FA08BD40
:10B4B000F8B54A002B4B520DD6182B4A0C460546C0
:10B4C000142E2BDA002E12DA284BFAF7EFF90022AD
:10B4D000134600F0F7FD40D2002C03DA0124E40704
:10B4E00000253AE02046284337D0214C14E0214F74
:10B4F0000B46F7403B402B4331D01C4BFAF7D6F9B3
:10B500000022134600F0DEFD27D2002C03DD0120CF
:10B510000005F0400419BC4300251EE0332E1EDC5C
:10B5200033460027143BFF43DF40384217D00F4B10
:10B53000FAF7D4F90022134600F0C4FD0DD2002C16
:10B540000ADD142E0CD03420811B012088404019C4
:10B55000A84200D2641C0546BD4321462846F8BDDA
:10B56000641CF9E701FCFFFF9C7500883CE4377E12
:10B570000000F03FFFFF0F007D2110B5C9004843D8
:10B5800000F001F810BD002140E000BF00BF00BF87
:10B5900000BF00BF00BF00BF00BF00BF00BF00BFB3
:10B5A00000BF00BF00BF00BF00BF00BF00BF00BFA3
:10B5B00000BF00BF00BF00BF00BF00BF00BF00BF93
:10B5C00000BF00BF00BF00BF00BF00BF00BF00BF83
:10B5D00000BF00BF00BF00BF00BF00BF00BF00BF73
:10B5E00000BF00BF00BF00BF00BF00BF00BF00BF63
:10B5F00000BF00BF00BF00BF00BF00BF00BF00BF53
:10B6000000BF00BF00BF00BF00BF491C8142BCD3C8
:10B6100070470000FEB5044600200190009060795C
:10B62000734940000E5A61782578491E7148CFB29F
:10B630000163042D77D0072D75D000210291217868
:10B6400001736C49E379012292058969002B6CD062
:10B65000914381616748217A4173217A8269890720
:10B66000890B0A4382610021042000F034FB32463A
:10B6700061492E2000F024FB3846FFF765FE5F4E3F
:10B680000522705D810040185D49431807212B2079
:10B6900000F030FB5B49029801220B180B21282097
:10B6A00000F028FB705D584980000A580C212820C2
:10B6B00000F011FBE079554980004018A17949005C
:10B6C000425A0221272000F0FBFA51487E00825B9B
:10B6D0000421272000F0F4FAE079002829D0A0788E
:10B6E00004282CD028206946087220220621272011
:10B6F00000F0E6FA02AB01222621272000F0FAFA38
:10B70000444938014018E17889004258082127202F
:10B7100000F0E1FAA17A601C627A0902114313D0A9
:10B7200016E000E001E0012188E71143F60881619D
:10B7300090E764220621272000F0C2FAE0E71020FB
:10B74000694608720246D1E733490172090A41721B
:10B75000417A007A0A0202432021272000F0B0FA41
:10B760002E4F0C2123203A6800F0B5FAF019828898
:10B770000421232000F0A4FAA07900280BD0E0795E
:10B780002749012243180021212000F0B3FA0320A9
:10B790000190012000902A07120F100102436078E7
:10B7A00000218007000B0243019800050243009826
:10B7B000400402432079C006400902436079C00674
:10B7C00002431F2000F087FAA07861780123084324
:10B7D00002040848DB030261E179490319430A4383
:10B7E00002610021082000F076FA0020FEBD000072
:10B7F0004CC300087001002004280000F4C20008B7
:10B800000C0000202A000020FCC200081CC3000815
:10B8100028C300082CC300084110000014C300080E
:10B820002C00002038B50C4607498A8B00210243C2
:10B830002C2000F045FA684604706B460122062170
:10B840002C2000F057FA38BD7001002010B5FFF72A
:10B8500067FD10BD10B504460421362000F0FCF849
:10B860000121C902002C01D0084300E088430246B0
:10B870000421362000F02FFA10BD000038B540201A
:10B880006946087000210E2000F0E6F80446002208
:10B8900011460E2000F01FFA6B46012200210D20F8
:10B8A00000F028FA074A00210F2000F014FA00F0F7
:10B8B000EDF9224600210E2000F00DFA0248002189
:10B8C000017338BDF8FF272490010020FEB505461E
:10B8D000042069460870514C0020607521462031D3
:10B8E000206348710873A0836063A06300F0C8F808
:10B8F0004B4E206002E000F0C3F82060B042FAD165
:10B900000020FFF73FFD00F0BBF8464E2060307886
:10B91000242801D9243806E00621F9F75CFD062227
:10B92000101A40010843020601040A4301020A43B7
:10B930000243B260706000211E2000F0CCF900F0DC
:10B940009FF820606B4601220021242000F0D2F9EC
:10B950001E20FFF78BFD86B2300AA0730420FFF78C
:10B9600085FD074600F08CF820603806000E0DD0EB
:10B9700002206946087101AB012212212D2000F03E
:10B98000B9F9A08B012109030843A08300F078F8DE
:10B9900020600620FFF76AFD60600720FFF766FD64
:10B9A000A060F006C00E207501D110202075C0B235
:10B9B00000F0DCF9E80707D0FFF73FFDA08B01217D
:10B9C000C9020843A0830AE00521362000F02EF8C2
:10B9D0001549084002460521362000F071F9012082
:10B9E000FFF7D0FC0021042000F036F8A061002110
:10B9F000262000F031F81521890308430246002172
:10BA0000262000F068F900222621362000F058F99F
:10BA100000F036F820600020FEBD0000700100201C
:10BA20003001CADE00000020FFFD000038B5094CDF
:10BA300089B280B26B46022200F028F8002806D1B5
:10BA400068464078010268460078081884B22046AB
:10BA500038BD0000FFFF000038B50024E44389B280
:10BA600080B26B46042200F011F8002806D10321B1
:10BA70006846435C2202D418491EFAD5204638BDD8
:10BA800010B500210846FFF7E7FF10BD38B50029C3
:10BA900009D0402420436C462070C8B27F2906D8C4
:10BAA000607002200AE069460870012006E08024E8
:10BAB00020436C466070C809A0700320694600F0FE
:10BAC000A1FA38BD10B5144603460A462146112096
:10BAD000FFF7DCFF10BD10B503460522002115203D
:10BAE000FFF7D4FF10BD10B5034605220021172033
:10BAF000FFF7CCFF10BD38B5054600206946087039
:10BB000000F0C4F8FF2401342246002D01D00322A6
:10BB1000120200210D2000F0D3F8002D13D06B4647
:10BB2000012203210F20FFF7B1FF684600780007CC
:10BB300009D5FFF7A3FE224600210D2000F0C0F832
:10BB40000020C04338BD002038BD10B50246012199
:10BB50000A2000F0C0F810BD10B5044600211A20DC
:10BB6000FFF77AFF000D22030005120B02430021AC
:10BB70001A2000F0B0F810BD10B5024602492E2080
:10BB800000F09EF810BD000004180000F8B505464E
:10BB90006B46012203210420FFF778FF0126114C98
:10BBA0003607002D0DD02A4600210C2000F088F821
:10BBB000694608781021084369460870A069304337
:10BBC00007E069460878EF21084069460870A069D7
:10BBD000B0430B46A06101220321042000F08AF843
:10BBE000F8BD00007001002010B5024600211820A9
:10BBF00000F066F810BD0000F8B50746002568465D
:10BC00000570B807204C2E4600280ADA80206946C5
:10BC100008706B46012200210D2000F06BF8012016
:10BC20002073F8076946087821D006210843694641
:10BC300008706B46012200210D2000F05BF8032103
:10BC40000F20FFF7F3FE8121C900084219D04020E0
:10BC5000694608706B46012200210D2000F04AF869
:10BC60000020FFF7F7FD00252673ED4309E00221D0
:10BC70000843694608706B46012200210D2000F040
:10BC800039F82846F8BD0000900100201CB56B462D
:10BC9000012203210F20FFF7F9FE684600784022B9
:10BCA000C1091040C9014000814208D00120694605
:10BCB0000871024601AB03210D2000F01BF81CBDEA
:10BCC00008B56B461A70120A5A7089B280B2022205
:10BCD00000F010F808BD38B500236C46E254120A93
:10BCE0005B1C042BFADB89B280B22346042200F0ED
:10BCF00001F838BD38B58024002909D0C025284373
:10BD00006D462870C8B27F2907D86870022009E004
:10BD1000204369460870012004E020436870C80988
:10BD2000A8700320694600F0A9F938BD10B5144683
:10BD3000012312189B029A4202D90020C04310BD71
:10BD40000B46821E21460920FFF7D4FF002010BDBC
:10BD500010B5054A8905126901430A4300210820EC
:10BD6000FFF7B9FF002010BD7001002038B5044670
:10BD70006B4601220E212B20FFF788FE68460078D3
:10BD8000E10640094001C90E0143684601706B4657
:10BD900001220E212B20FFF7ADFF38BD10B5002189
:10BDA00042541C06120A22431B0A491C0429F7DBD1
:10BDB00010BD7CB5002425466846FFF78CFE0420A4
:10BDC0006946220E2D02154322020C5C1443401ECC
:10BDD000F7D5204629467CBD7CB50024254668461B
:10BDE000FFF781FE04206946220E2D021543220230
:10BDF0000C5C1443401EF7D5204629467CBD00004C
:10BE0000FBF702FCFEF7F8FBFDF7E8FAFDF7FAFA9C
:10BE10003A493B48002522C005608561C561394922
:10BE20000562C1600838FBF773FDFDF7F5FBFDF710
:10BE30008FFBFDF79FFAFDF7ADFB052401222407D8
:10BE4000D1032046FBF7CBFBFEF788F9FDF778F925
:10BE5000FAF75EFCFAF72CFC0721A015FFF7E2FCCD
:10BE6000FFF7F4FC012211032046FBF7B8FB24483E
:10BE7000C8222549C830FCF7FBFE244F244E254C30
:10BE8000387800280DD1A06A4000000E09D1402169
:10BE90003046FBF797FB002803D101210846FBF74A
:10BEA00057FE2079002826D06078002823D02571FD
:10BEB00072B620780F2808D901200003B061FEF780
:10BEC000E9FC01200003B0620CE00122510330467E
:10BED000FBF785FBFEF7DEFC01210022490330461B
:10BEE000FBF77DFB62B6FDF74BF8208C0028C7D02E
:10BEF000401E2084C4E7FDF743F8C1E7007C004002
:10BF0000B8150020FFFF0000D40C002042000020E4
:10BF1000000400502401002010B586B0FDF7BEF8E3
:10BF20001748FBF778FC14216846F9F752FA1548D0
:10BF30000090032001900020029005206946000730
:10BF4000FBF768FA69461048FBF764FA69460F4840
:10BF5000FBF760FA01210846FBF7FAFDFF240134E4
:10BF60002046FBF7CDFD0A4908680422104308600B
:10BF70002046FBF7D5FDFBF7DBFD06B010BD00004A
:10BF8000B8150020FFFF000000040050000800501A
:10BF90000070004010B50122920216491648FAF7C7
:10BFA00031FC1448154902888A4222D00180144984
:10BFB0008180FF21F531C1800A21018100211E22EB
:10BFC0004181D24382810122C28181834323C3867E
:10BFD0000287782343878287C287024640321184D2
:10BFE00051849184C183918014238382118200F053
:10BFF0002FF810BD9C0D002000FC0008AA55000081
:10C0000034120000F0B58C460025102605210907E2
:10C010008E620E4C08E067467F5DE760A768FF0709
:10C02000FCD0E7681F706D1C8542F4DB00200746DA
:10C0300006E0E760A568ED07FCD0E5681D54401CEC
:10C040009042F6D38E610020F0BD00000030014028
:10C0500070B572B60124074DA40221462846FAF7AE
:10C06000B7FB002804D0224603492846FAF754FCBF
:10C0700062B670BD00FC00089C0D0020F0B50025E4
:10C08000102605279C463F070B46BE620C4C06E077
:10C09000595DE160A168C907FCD0E1686D1C85426B
:10C0A000F6DB002007E06146095CE160A168C90792
:10C0B000FCD0E168401C9042F5D3BE610020F0BD89
:10C0C0000030014070B501251C002D050C4310D433
:10C0D000EC4206D4AC420AD48B4200D070BD8242FE
:10C0E00070BDEB4217D4E94215D48B4270BD9B4220
:10C0F00070BDEC4206D5AC42F9D5994200D070BD76
:10C10000904270BD6D005C00EC4204D24C00EC42E9
:10C1100001D2994270BD0FB4034C0CBC03BC30B4C7
:10C12000FAF7E4F830BC70BD1900160470B50125AB
:10C130000400ED074C4020D4441A01D2001B091919
:10C14000C60D4B00F2B2FF2A29D01B0E2CD00002E4
:10C150000C02D31A2C43DC402843051910D2280ABC
:10C1600002D3401C6D0611D0761EF6058019FF2AF9
:10C1700000DA70BDC00DC00570BD694000F058F810
:10C1800001200543C541521C761CE8E764089C4029
:10C19000C90161408900E7D10124A043E4E71B0EF7
:10C1A000440200D0034870BD002AFCD1C00FC00774
:10C1B00070BD00BF0000C07F01230200DB050A4301
:10C1C0000DD4DA4203D49A4207D488427047D84249
:10C1D00014D4D94212D48842704780427047DA4260
:10C1E00003D59A42F9D5814270475B004200DA429A
:10C1F00004D24A00DA4201D28142704710B5024AA5
:10C20000FAF7BCF810BD00BF0900160470B501258F
:10C21000ED07684004004C4002D5694000F008F882
:10C22000FFF78AFF70B501250400ED074C4022D4CA
:10C23000441A02D26C40001B0919C60D4B00F2B221
:10C24000FF2A4BD01B0E50D000020C02D31A2C43F5
:10C25000DC40A843051B05D5AD0019D36D08761E3B
:10C26000521E37D0F605280A01D2801970BD7041E0
:10C270006D0603D070BD6940FFF75EFF9C40090268
:10C280006140490001D0401E70BD0124A04370BD33
:10C290006D081DD001202B0C01D12D0410302B0E68
:10C2A00001D12D0208302B0F01D12D01001DAB0F44
:10C2B00001D1AD00801CEB0F01D16D00401C6D0061
:10C2C000361A121A680AF5054019012A02DB70BDF8
:10C2D000002070BDC036300AC00770BD1B0E44027E
:10C2E00001D1FF2B00D1024870BD002AF0D070BDF3
:10C2F0000000C07F0000010203040005405C000054
:10C30000A05C0400C06C0800805C0400E03F1E00DC
:10C31000E07D1E0007A9022570889B880A00160090
:10C32000010006000100020087008D002D001A3177
:10C3300052001A339A001A351D011A376B003B312F
:10C34000BE003B335E013B3596023B3700009959F6
:10C350009959EB518F421E45142E0080EB51F52860
:10C360003333E13A703DE13AC235852BC235333380
:10C37000C235C235AE47E13A5138A33051380000DA
:10C38000000000000000010203040607080903047E
:10C3900006080C1018203000000000010203048081
:10C3A000807F7E7D7C7B7A79787776767574737200
:10C3B0007171706F6E6E6D6C6C6B6A6A69686867BC
:10C3C0006666656464636362616160605F5F5E5E50
:10C3D0005D5D5C5C5B5B5A5A5959585857575656C5
:10C3E0005555555454535352525251515050504F29
:10C3F0004F4F4E4E4D4D4D4C4C4C4B4B4B4A4A4A79
:10C4000049494948484847474747464646454545BC
:10C4100044444444434343434242424241414181B4
:10C4200082838485868788898B8C8D8E8F91929369
:10C43000959697999A9C9D9FA0A2A3A5A7A8AAAC00
:10C44000AEB0B2B3B5B7B9BCBEC0C2C5C7C9CCCE19
:10C45000D1D4D7D9DCDFE2E6E9ECF0F3F7FAFE005D
:10C4600080C400080000002070010000F66400088D
:10C47000E4C4000870010020A01C00000451000862
:10C48000C1130704380D091E08054008260910408D
:10C4900008560A131D043B08BE0516D8BC401008F8
:10C4A0005201033AC842077052030CE5800C1B028C
:10C4B00002DD140901022281F01F66810498899629
:10C4C000869679821598039814988796749778823F
:10C4D000439788967197778249F10139293F9204F1
:04C4E0001220000026
:04000005080050C1DE
:00000001FF
